:100000000C94B2070C94DA070C94DA070C94DA0714
:100010000C94DA070C94DA070C94DA070C94DA07DC
:100020000C94DA070C94DA070C940A1A0C94791AD7
:100030000C94DA070C94DA070C94DA070C94DA07BC
:100040000C94DA070C94DA070C94DA070C94DA07AC
:100050000C94DA070C94DA070C94DA070C94AB1CB6
:100060000C94DA070C94DA070C94DA070C94DA078C
:100070000C94DA070C94DA070C94DA070C94DA077C
:100080000C94DA070C94DA070C94DA070C94DA076C
:100090000C94DA070C94DA070C94DA070C94DA075C
:1000A0000C94DA070C94DA070C94DA0744617900AF
:1000B00041636374004C6F616E00436170616369FA
:1000C0007479200053707261792000050512151FA4
:1000D000150905082466E766244120596573202028
:1000E00042204E6F000043616E6479204361737457
:1000F0006C6500536F6461205377616D70004775C4
:100100006D6D7920466F726573740043686F636F1D
:100110006C616E640049636520437265616D2052B5
:1001200064005377656574205375697465730000C6
:100130004C6F6C6C7900536F757273004D61727304
:10014000004165726F004865727368657900502ED2
:100150005375676172002000200003081F051F1FF0
:10016000151B1F11111F110E1F15111F05011F1146
:100170001D1F041F001F0010101F1F041B1F101045
:100180001F061F1F011F1F111F1F05071F311F1FE4
:10019000051B17151D011F011F101F0F100F1F0C2E
:1001A0001F1B041B071C071915130C121E1F120C12
:1001B0001E12120C121F0C1A14041F052E2A1E1FC9
:1001C000021C001D00201D001F041A011F001E0438
:1001D0001E1E021E1E121E3E120C0C123E1E020697
:1001E00014120A020F121E101E0E100E1E081E1AE6
:1001F000041A2E281E1A12161F111F001F001D158B
:100200001711151F07041F17151D1F151D01011FAD
:100210001F151F17151F00170000100020100000E9
:10022000030004083E09093E3F25251A1E2121121C
:100230003F21211E3F2525213F0505011E21293A89
:100240003F04043F213F21001021211F3F040A31B8
:100250003F2020203F02023F3F02043F1E21211E7B
:100260003F0909061E21112E3F09093622252519AD
:10027000013F01011F20201F0F10201F3F10103FC2
:100280003B04043B03043807312D2321102A2A3C68
:100290003F2424181C2222141824243F1C2A2A2C10
:1002A000047E05014C52523E3F040438243D200098
:1002B0004040443D3F081422213F20003E04043EBC
:1002C0003E04023C1C22221C7E22221C1C22227E76
:1002D0003E040204242A2A12021F22201E20201E6D
:1002E0000E10201E3E10103E360808364E50503E6E
:1002F000322A26221E29251E223F200032292926A5
:100300001221251A0C0A3F08172525191E25251824
:10031000013905031A25251A0629291E002F000078
:10032000002000004020000000030000000000004A
:10033000003E5B4F5B3E3E6B4F6B3E1C3E7C3E1C6B
:10034000183C7E3C181C577D571C1C5E7F5E1C00B1
:10035000183C1800FFE7C3E7FF0018241800FFE768
:10036000DBE7FF30483A060E2629792926407F052B
:100370000507407F05253F5A3CE73C5A7F3E1C1C41
:1003800008081C1C3E7F14227F22145F5F005F5F01
:1003900006097F017F006689956A606060606094ED
:1003A000A2FFA29408047E040810207E20100808F2
:1003B0002A1C08081C2A08081E101010100C1E0CFD
:1003C0001E0C30383E3830060E3E0E06000000008F
:1003D0000000005F00000007000700147F147F1476
:1003E000242A7F2A122313086462364956205000BB
:1003F00008070300001C2241000041221C002A1CA7
:100400007F1C2A08083E0808008070300008080891
:100410000808000060600020100804023E514945B1
:100420003E00427F400072494949462141494D33CF
:100430001814127F1027454545393C4A4949314136
:10044000211109073649494936464949291E000004
:100450001400000040340000000814224114141459
:100460001414004122140802015909063E415D5945
:100470004E7C1211127C7F494949363E414141224E
:100480007F4141413E7F494949417F090909013E78
:10049000414151737F0808087F00417F410020409F
:1004A000413F017F081422417F404040407F021CB1
:1004B000027F7F0408107F3E4141413E7F090909C8
:1004C000063E4151215E7F09192946264949493294
:1004D00003017F01033F4040403F1F2040201F3F5A
:1004E0004038403F631408146303047804036159DF
:1004F000494D43007F414141020408102000414121
:10050000417F0402010204404040404000030708CC
:100510000020545478407F284444383844444428C8
:10052000384444287F385454541800087E0902186F
:10053000A4A49C787F0804047800447D40002040F7
:10054000403D007F1028440000417F40007C04783B
:1005500004787C080404783844444438FC18242483
:100560001818242418FC7C08040408485454542403
:1005700004043F44243C4040207C1C2040201C3C80
:100580004030403C44281028444C9090907C446477
:10059000544C44000836410000007700000041360A
:1005A000080002010204023C2623263C1EA1A16190
:1005B000123A4040207A38545455592155557941C2
:1005C0002154547841215554784020545579400C99
:1005D0001E5272123955555559395454545939557A
:1005E0005454580000457C410002457D42000145BD
:1005F0007C40F0292429F0F0282528F07C5455452A
:10060000002054547C547C0A097F493249494932BC
:100610003248484832324A4848303A4141217A3AD1
:1006200042402078009DA0A07D39444444393D409B
:1006300040403D3C24FF2424487E4943662B2FFC48
:100640002F2BFF0929F620C0887E090320545479F6
:10065000410000447D413048484A32384040227AC7
:10066000007A0A0A727D0D19317D2629292F282644
:100670002929292630484D4020380808080808084C
:100680000808382F10C8ACBA2F102834FA00007BA5
:10069000000008142A142222142A140895002200AB
:1006A00095AA005500AAAA55AA55AA000000FF0065
:1006B000101010FF00141414FF001010FF00FF10A2
:1006C00010F010F0141414FC001414F700FF0000D4
:1006D000FF00FF1414F404FC141417101F10101F53
:1006E000101F1414141F00101010F0000000001F41
:1006F000101010101F10101010F010000000FF104C
:100700001010101010101010FF10000000FF140047
:1007100000FF00FF00001F10170000FC04F4141479
:100720001710171414F404F40000FF00F714141445
:1007300014141414F700F7141414171410101F10C5
:100740001F141414F4141010F010F000001F101FE8
:100750000000001F14000000FC140000F010F01056
:1007600010FF10FF141414FF141010101F000000CD
:1007700000F010FFFFFFFFFFF0F0F0F0F0FFFFFFD1
:100780000000000000FFFF0F0F0F0F0F3844443828
:10079000447C2A2A3E147E02020606027E027E0263
:1007A00063554941633844443C04407E201E200682
:1007B000027E020299A5E7A5991C2A492A1C4C72BF
:1007C00001724C304A4D4D303048784830BC625A46
:1007D000463D3E494949007E0101017E2A2A2A2AD6
:1007E0002A44445F444440514A444040444A5140B2
:1007F0000000FF0103E080FF000008086B6B083673
:1008000012362436060F090F0600001818000000E3
:100810001010003040FF0101001F01011E00191DD2
:100820001712003C3C3C3C0000000000D5F08D1449
:10083000A1C881CFD9F1AF2000F0F89C8E878387C3
:100840008E9CF8F00000FEFF0303030303070EFC79
:10085000F80000FEFF0303030303070EFCF800008B
:10086000FFFF00000000000000FFFF0000FEFF830C
:1008700083838383C7EE7C380000F8FC0E070303F4
:1008800003070EFCF800003F7FE0C08080C0E07FDF
:100890003FFFFF01010101010101FFFF0000FFFF18
:1008A0000C0C0C0C1C3E77E3C100007FFFC0C0C0E5
:1008B000C0C0E0703F1F00001F3F70E0C0C0C0E03C
:1008C000703F1F00007FFFC1C1C1C1C1E3773E1C63
:1008D00000001F3F70E0C0C0C0E0703F1F0000007C
:1008E000000001FFFF01000000647572696E67205F
:1008F0007468652063686173652121006275636BAC
:10090000732066726F6D2070757273657300596F16
:100910007520736E6174636865642000546865793E
:1009200020616C6C20676176652075702100412024
:100930004D6F6D2067617665207570212100002064
:1009400020596F75206D6973736564212121000042
:100950006861766520746F2072756E2100616E7912
:100960002073707261792120596F7500596F75205D
:10097000646F6E27742068617665007468656D2108
:1009800000596F752063616E2774207368616B6511
:1009900000616E20616C6C6579212100596F7520B2
:1009A0006C6F7374207468656D20696E00756E6974
:1009B0007473206F663A2000596F7520666F756EEC
:1009C000642000323030206275636B733F006D6FBE
:1009D000726520737061636520666F720063616E7B
:1009E0006479207361636B20776974680057696C60
:1009F0006C20796F75206275792061206E657700B3
:100A000057696C6C20796F75206561742069743F3B
:100A1000006D6F73746C7920756E636865776564BB
:100A2000212100686572652074686174206C6F6FA5
:100A30006B73005468657265277320736F6D652052
:100A400067756D00646F6C6C6172733F00737072D8
:100A5000617920666F7220343030004D6F6D2072E6
:100A60006570656C6C616E74007374696E6B207375
:100A70007072617920666F7200736C6565702073A7
:100A80007072617920666F720034303020646F6C50
:100A90006C6172733F0057696C6C20796F752062CE
:100AA0007579206100616674657220796F75210027
:100AB000667269656E64732061726500206F6620DE
:100AC00068657200616E642000596F7572204D6F09
:100AD0007468657200746F2063686172697479214B
:100AE00000596F7520676176652061206269740026
:100AF000617265206F7574726167656F757321210E
:100B000021210073686F72746167652120507269DA
:100B100063657300506F77646572656420737567F1
:100B20006172007072696365732121210061742014
:100B30006F7574726167656F757300627579696E40
:100B40006720486572736865790043686F636F68F2
:100B50006F6C696373206172650062616B652D6FF4
:100B60006666212121210066726F6D206C617374AD
:100B7000207765656B277300636865617020486541
:100B80007273686579004D6F6D73206172652073B3
:100B9000656C6C696E6700626F74746F6D6564205C
:100BA0006F7574212121004D617273207072696329
:100BB00065732068617665006C6F6C6C792121210A
:100BC000006172652073656C6C696E67206368658F
:100BD0006170004B696473206174207363686F6F88
:100BE0006C00746F6461792100626F72726F776557
:100BF00064206D6F6E657900596F7520616C726548
:100C0000616479002100596F7520646F6E2774202C
:100C10006861766520616E7900004F6F7073210006
:100C20002100596F752063616E2774206166666FBD
:100C3000726400004F6F7073210021006D6F726548
:100C40002000596F752063616E2774206361727292
:100C50007900004F6F70732100596F7527726520FE
:100C60006361756768742121006265656E2068693B
:100C7000742100596F75277665006D69737365641B
:100C80002121005468657900796F75212120005475
:100C9000686579277265206E616767696E670041D4
:100CA0002053707261792020422052756E004552A7
:100CB000524F522000416D7400536176696E677324
:100CC00000596F75206F776500596F7520686176E0
:100CD00065005769746864726177204D6F6E65793D
:100CE000004465706F736974204D6F6E65790042C2
:100CF0006F72726F77204D6F6E6579005061792049
:100D00004C6F616E00000051747900507269636528
:100D100000436F73747300596F75206861766500C6
:100D200053656C6C200042757920000000796F7566
:100D3000722074656574683F0064656E74697374CD
:100D400020746F2066697800646F6C6C6172732028
:100D5000666F7220610057696C6C20796F75207026
:100D60006179203130303000596F757220686561CB
:100D70006C74683A20007374696C6C2061667465E9
:100D80007220796F752100204D6F6D730054686576
:100D900072652061726520004265696E6720636834
:100DA00061736564212100576974686472617720FA
:100DB0004D6F6E6579004465706F736974204D6F77
:100DC0006E65790042616E6B00426F72726F7720C0
:100DD0004D6F6E6579005265706179204C6F616E60
:100DE0000052696368204275646479004A65742022
:100DF00066726F6D200053656C6C2043616E647980
:100E0000004275792043616E64790043616E6479B4
:100E1000205361636B0042616E6B0052696368200E
:100E20004275646479004A65740043616E64792098
:100E30005361636B0053656C6C2043616E64790091
:100E40004275792043616E64790048697420746842
:100E500065205374726565747321210076312E31DB
:100E60002E310043616E6479576172001E1E0000CE
:100E70000000000000000000000000C0F0E8C48294
:100E800002033F3F0F8782C2C4C8F0C000000000C9
:100E90000000008080807088A80FF1810181C1E18D
:100EA000F0FCF000818143271F0700000000008054
:100EB00040A1562C1434224176080D090701010186
:100EC00001010000000000003028140A05020100A2
:100ED0000000000000000000000000000000000012
:100EE000000000000000080B0002020200000904DC
:100EF0000000010202000005240010010524010188
:100F000001042402060524060001070581031000E0
:100F10004009040100020A00000007050202400027
:100F200000070583024000000403090412010002C7
:100F3000EF020140412336800001010203014172AA
:100F40006475696E6F204C4C430041726475696E24
:100F50006F204C656F6E6172646F0003051F0E0495
:100F6000281DC92F11241FBECFEFDAE0DEBFCDBF91
:100F700012E0A0E0B1E0E2E5FDE602C005900D92CE
:100F8000A036B107D9F727E0A0E6B2E001C01D9274
:100F9000A03AB207E1F717E0C1EBD7E004C0219710
:100FA000FE010E94A434C03BD107C9F70E94A91DCD
:100FB0000C949C360C940000E2EFF2E0A0E0B8E064
:100FC00000800EBC8111012C1197A0FDFDCF019274
:100FD000B9F70DB40895480F592F511D1416150671
:100FE00084F5803891056CF597FF02C090E080E0B1
:100FF0004138510514F040E850E0481BFB01E77010
:10100000FF2721E001C0220FEA95EAF777FF02C02F
:10101000695F7F4FFB0133E0F595E7953A95E1F77E
:10102000F695FE2FEE27F795E795E80FF91FEE509E
:10103000FD4F415030F08191DF011197822B8C934D
:10104000F8CF08956F927F928F929F92AF92BF9246
:10105000CF92DF92EF92FF920F931F93CF93DF9384
:10106000DC01FA011491319654913196C12FD0E0F0
:10107000222309F1CC24C394D12C852F877011F43D
:10108000D12CC12CE52EE694E694E694EC0CFD2CD4
:10109000F11CEC9EC001ED9E900DFC9E900D112464
:1010A000033011F4880F991F289F7001299FF00CBD
:1010B0001124EE0DFF1D7D01EC0EFD1E1E141F04FC
:1010C0000CF06BC0A038B1050CF067C0CB01850FE8
:1010D000911D181619060CF060C0603471050CF0F3
:1010E0005CC0309709F459C0362F3770CB0177FDBB
:1010F000079623E0959587952A95E1F7282F77FFA6
:1011000004C0332311F02FEF280F662777276A1BBF
:101110007B0BB7FD02C070E060E090E89A1B40E8EE
:10112000E416F1040CF4912F961BE22E022E000C13
:10113000FF08DE2CD0942F3F0CF0D12C41E0852FFE
:10114000877009F440E0B52EB694B694B6944B0D72
:10115000E40EF11C89E0E816F10414F048E0421BAB
:10116000B42EBD182D0D40E8240370011124AE0DDE
:10117000BF1DA60FB71F1D9D600D711D1124AF016E
:10118000460F571FC32E032E000CDD08033009F451
:10119000C7C090F4023009F474C0DF91CF911F9161
:1011A0000F91FF90EF90DF90CF90BF90AF909F9006
:1011B0008F907F906F9008950A3FA1F1B20E0B3F80
:1011C00061F72B1551F3BD016E507D4F10E000E02B
:1011D000091708F09FC0FA01E00FF11FE491F0E059
:1011E0004F010C2C02C0880C991C0A94E2F727FDD1
:1011F00006C0FB018081F82CF0948F21808333237B
:1012000061F0273054F47B01F0E8EF0EF11CA92CBB
:10121000A094F70180818A2180830F5F1F4F6F5F49
:101220007F4FD6CFB20E2B1509F4B7CFBD016E504C
:101230007D4F10E000E0091708F066C0FA01E00FEA
:10124000F11FE491F0E04F010C2C02C0880C991CB6
:101250000A94E2F727FD04C0FB018081882980837E
:10126000332351F0273044F47B01F0E8EF0EF11CFA
:10127000F7018081892980830F5F1F4F6F5F7F4F48
:10128000DACF6FEF70E0032E02C0660F771F0A946B
:10129000E2F760957095972E8B2C820E281509F435
:1012A0007CCF8D010E501D4FF12CE12CE91630F54D
:1012B000FA01EE0DFF1DE491F0E03F010C2C02C09D
:1012C000660C771C0A94E2F727FD05C0F8018081BF
:1012D000862386298083332359F027304CF4580124
:1012E000F0E8AF0EB11CF501808189218729808348
:1012F000FFEFEF1AFF0A0F5F1F4FD8CF2F5F4C0F82
:101300005D1FA058BF4FCACF2F5F4C0F5D1FA05865
:10131000BF4F89CF2F5F4C0F5D1FA058BF4F51CFDC
:10132000E92EF12CFA01E60FF71FAE50BD4F60E831
:1013300070E06E197F09CE19DF098E01000F111FB1
:1013400041E050E07A01032E01C0EE0C0A94EAF766
:10135000592F4B2D892E932ECF93DF93ED01EF96CE
:10136000EF962296A590C590992059F0AE9C500119
:10137000CE9C600127302CF4F880D094FD20FB280F
:10138000F99222233AF0FC90C094FC20FA28FD92B6
:101390000C94CB0911965A9529F74A9551F0582D7E
:1013A00023951124E00FF11DA60FB11DC60FD11D0D
:1013B000D9CFDF91CF911124F0CE0F9302E020E03E
:1013C0000E9422080F9108952F923F924F925F92B0
:1013D0006F927F928F929F92AF92BF92CF92DF9245
:1013E000EF92FF920F931F93CF93DF93CDB7DEB7AA
:1013F00028970FB6F894DEBF0FBECDBF6F836A018A
:1014000019011C830B83FE82ED82811128C005E047
:1014100010E029E030E03A832983B6010D2C000C5E
:10142000880B990B0E9408314B015C015F815111BF
:101430001DC0E0E6F7E090E080E018861F828C1582
:101440009D050CF02BC1248135814F8158854217B1
:10145000530714F438872F8301963696F0CF04E0B3
:1014600010E048E050E05A834983D7CF20E030E0D5
:1014700040E05FE30E9467314B015C0120E030E017
:10148000A9010E94423420E030E040E05FE387FDA4
:1014900030C0C501B4010E94D6320E94B4337887AF
:1014A0006F83A6018F819885481B590BE0E6F7E012
:1014B00090E080E0B12CA12C2F8138858217930712
:1014C000ECF086E0829FF001839FF00D1124E05A3A
:1014D000F84F90E080E0D12CC12C84179507BCF424
:1014E00024813581C216D3060CF469010196369623
:1014F000F4CFC501B4010E94D532CFCF248135810C
:10150000A216B3060CF4590101963696D5CFB80150
:10151000110F880B990B0E9408312B013C01B5017A
:101520006C0D7D1D072E000C880B990B0E94083155
:1015300020E030E040EE5FE30E94D6326B017C0198
:1015400020E030E040E05FE3C301B2010E94673178
:101550009B01AC01C701B6010E9467316B017C01A0
:1015600020E030E0A9010E94423420E030E040E079
:101570005FE387FD89C0C701B6010E94D6320E9491
:10158000B43302E410E0061B170BF1011183008352
:10159000B501BB0C880B990B0E94083120E030E0AC
:1015A00040EE5FE30E94D632A30192010E946731B0
:1015B0004B015C0120E030E0A9010E94423420E0B0
:1015C00030E040E05FE387FD64C0C501B4010E94E4
:1015D000D6320E94B433600F711FEB81FC8171839E
:1015E000608329813A81B901330F880B990B0E94DE
:1015F000083120E030E040E05FE30E9467316B019A
:101600007C014F815885BA01550F880B990B0E94B8
:1016100008319B01AC01C701B6010E9467316B0123
:101620007C0120E030E0A9010E94423420E030E05B
:1016300040E05FE387FD85C0C701B6010E94D63256
:101640000E94B4332AE230E0C901861B970BED817A
:10165000FE819183808328960FB6F894DEBF0FBE7B
:10166000CDBFDF91CF911F910F91FF90EF90DF9051
:10167000CF90BF90AF909F908F907F906F905F9032
:101680004F903F902F900895C701B6010E94D53228
:1016900076CFC501B4010E94D5329BCFB801110F9E
:1016A000880B990B0E94083120E030E040E05FE3B6
:1016B0000E9467312B013C01EF81F885BF01FF0FCC
:1016C000880B990B0E9408319B01AC01C301B20148
:1016D0000E9467312B013C0120E030E0A9010E940B
:1016E000423420E030E040E05FE387FD25C0C301E5
:1016F000B2010E94D6320E94B43322E430E0C90124
:10170000861B970BF101918380838FEF9FEFEB8115
:10171000FC819183808329813A81B901330F880B41
:10172000990B0E94083120E030E040E05FE30E9426
:101730006731A501940171CFC301B2010E94D53276
:10174000DACFC701B6010E94D5327ACFFC01809171
:10175000F102882311F13FB7F89482E08093E90009
:101760002091F200822F90E01816190614F481E0FF
:1017700090E0882339F0289844E64093F0024091A5
:10178000F1004083222339F02091F200211103C09F
:101790002BE62093E8003FBF08958FEF9FEF089559
:1017A0002FB7F89483E08093E9009091E800892FA7
:1017B000807295FF04C09091F20080E4891B2FBFD6
:1017C00008958091E80281110DC082E08093E402C7
:1017D00084E08093E5021092E7021092E60281E035
:1017E0008093E80284EE92E00895CF93DF931F92F6
:1017F000CDB7DEB76983DC01ED91FC910280F38106
:10180000E02D41E050E0BE016F5F7F4F09950F90E2
:10181000DF91CF91089583E08093E9008091F200F9
:10182000882319F08AE38093E80008950E94D00B82
:1018300090E00895CF93DF931F92CDB7DEB7FC0100
:101840008485958597FD08C02FEF3FEF3587248766
:101850000F90DF91CF910895CE0101960E94A60BC3
:10186000019719F4898190E0F3CF8FEF9FEFF0CFCC
:101870000F931F93CF93DF931F92CDB7DEB78C01E9
:10188000FC018485958597FF0BC0CE0101960E94CF
:10189000A60B019771F4898190E0F8019587848700
:1018A000F801848595850F90DF91CF911F910F915D
:1018B00008958FEF9FEFF1CFFC018485958597FD0B
:1018C0000BC09FB7F89482E08093E9008091F2000A
:1018D0009FBF90E0019608959FB7F89482E08093AF
:1018E000E9008091F2009FBF90E008954091DE02F0
:1018F0005091DF022091DC023091DD024217530744
:10190000B4F49091E8009570E1F39091E80092FDB5
:1019100019C08093F1008091DE029091DF02019660
:101920008F739927892B19F48EEF8093E8008091AB
:10193000DE029091DF0201969093DF028093DE0237
:1019400081E0089580E00895DF92EF92FF920F9377
:101950001F93CF93DF93D82E8A01EB017B01E40E16
:10196000F51ECE15DF0559F0D7FE12C0FE01849199
:101970000E94760C21968111F4CF0FEF1FEFC80162
:10198000DF91CF911F910F91FF90EF90DF9008951D
:101990008881EECF0F931F93CF93DF931F92CDB724
:1019A000DEB782E0898342E450E066EE7EE080E8C4
:1019B0000E94A40C0E94E10BDC0112960D911C9177
:1019C0000115110589F0D801ED91FC910280F38198
:1019D000E02DBE016F5F7F4FC801099597FD04C0E0
:1019E000F80100851185ECCF89810F90DF91CF91AF
:1019F0001F910F910895615030F02091F100FC018A
:101A000020830196F8CF289884E68093F002089509
:101A10003FB7F8948091D8029091D902A091DA0250
:101A2000B091DB0226B5A89B05C02F3F19F00196A7
:101A3000A11DB11D3FBFBA2FA92F982F8827BC0128
:101A4000CD01620F711D811D911D42E0660F771F50
:101A5000881F991F4A95D1F708958F929F92AF9250
:101A6000BF92CF92DF92EF92FF926B017C010E94B6
:101A7000080D4B015C01C114D104E104F104B9F07B
:101A80000E94080D681979098A099B09683E73400C
:101A90008105910580F321E0C21AD108E108F1081F
:101AA00088EE880E83E0981EA11CB11CE4CFFF9045
:101AB000EF90DF90CF90BF90AF909F908F90089560
:101AC0008F929F92AF92BF92CF92DF92EF92FF924E
:101AD0000F931F93CF93DF936C017B018A01809159
:101AE0000C01882309F45CC08091F102882309F479
:101AF00057C08091E30280FF05C08091E0008260C2
:101B00008093E000E801B12C8AEFA82E93E0892EA3
:101B10002AE3922E209711F4BB20D9F10E94D00B1A
:101B200081110AC0AA94AA20D9F161E070E080E096
:101B300090E00E942D0DEECF8C171D0611F00CF0D9
:101B40008C2F9FB7F8948092E9002091E80025FD42
:101B500002C09FBFDFCF282F30E0C21BD30BF7019D
:101B6000815020F041914093F100FACFE20EF31E34
:101B7000BB2021F09092E800B12CEBCF8091E800DF
:101B800085FDE7CF9092E800BB24B394209709F33A
:101B9000F3CF5D9884E68093E202101611063CF0C4
:101BA00081E090E0F6019383828310E000E0C801B9
:101BB000DF91CF911F910F91FF90EF90DF90CF9029
:101BC000BF90AF909F908F9008950895DB01149679
:101BD0004D915C9115976D917C91DC01ED91FC919B
:101BE0000280F381E02D09942F923F924F925F92F1
:101BF0006F927F928F929F92AF92BF92CF92DF921D
:101C0000EF92FF920F931F93CF93DF9300D000D0FA
:101C100000D0CDB7DEB7782E662E5A0128E0422ECE
:101C2000512C811103C099E0492E512CCE0101960F
:101C30007C018E010D5F1F4F9E012B5F3F4FA50161
:101C4000662D872D0E94E409B5010B2C000C880B32
:101C5000990B0E94083120E030E040E05FE30E94F1
:101C600067316B017C0120E030E0A9010E94423421
:101C700020E030E040E05FE387FD24C0C701B6010B
:101C80000E94D6320E94B4338B0180E6C82E87E0D2
:101C9000D82E049D1001059D300C149D300C11248C
:101CA000F12CE12C912C812C8A149B04B4F58981B0
:101CB0009A81662019F0801691064CF42D818E0DC4
:101CC0009F1D0BC0C701B6010E94D532DBCF2B810F
:101CD000A70142195309840F951F7720A1F0209383
:101CE00089072093880780938A07B60184E897E0E4
:101CF0000E94E60D9FEF891A990A86E0C80ED11C52
:101D0000E40CF51CD1CF2093930720939207809386
:101D10009407B6018EE897E0EBCF26960FB6F894BD
:101D2000DEBF0FBECDBFDF91CF911F910F91FF900E
:101D3000EF90DF90CF90BF90AF909F908F907F906B
:101D40006F905F904F903F902F900895EF92FF9289
:101D50000F931F93CF93DF938C017B01D0E0C0E002
:101D6000F701EC0FFD1F6491662361F0D801ED913E
:101D7000FC910190F081E02DC8010995892B11F0AB
:101D80002196EECFCE01DF91CF911F910F91FF9061
:101D9000EF900895AF92BF92CF92DF92EF92FF92B1
:101DA0000F931F93CF93DF936C017B018B01040F83
:101DB000151FEB015E01AE18BF08C017D10759F01F
:101DC0006991D601ED91FC910190F081E02DC60161
:101DD0000995892B79F7C501DF91CF911F910F915B
:101DE000FF90EF90DF90CF90BF90AF9008952D9A25
:101DF0000895BC0190E080E00C942D0D8FB180958A
:101E0000807F669B88601C9B8460089581EC809332
:101E10007C0085B1806F85B984B1877E84B984B137
:101E2000876E84B95E9A5F988AB1806D8AB9769A16
:101E30006E9881B3806F81BB899880B38D7080BBB1
:101E400080E58CBD81E08DBD85E090E00E94F90EBB
:101E50005F9A85E090E00E94F90E5E985C98ECE253
:101E6000F8E084918EBD00000DB407FEFDCF3196E1
:101E700088E0E933F807A9F75C9A81E88093640069
:101E8000809165008160809365000895909168025B
:101E9000982329F490916902982381E009F480E065
:101EA0000895CF93C82F0E94FE0E982F9C2381E0A7
:101EB0009C1380E0CF91089580E00C94DC0780387B
:101EC0009105B8F460347105A0F420E191E061FD62
:101ED00094E060FD990F62FD9295687F269FD00186
:101EE0001124A80FAE50BD4F8C9140FF03C0892B29
:101EF0008C93089590958923FBCF2F923F924F9218
:101F00005F926F927F928F929F92AF92BF92CF9289
:101F1000DF92EF92FF920F931F93CF93DF937C0199
:101F20006B0188248394912CD0E0C0E005E010E0A0
:101F300096EF692E77247A942CEFA22EBB24BA94C4
:101F4000842F8470582E842F8270482E842F88709E
:101F5000382E4170242E219682E0880E911CA80C08
:101F6000B91C552091F041E0B8016C0D7D1DC701F1
:101F70008C0F9D1F0E945F0F41E0B6016C0F7D1F0B
:101F8000C8018E0D9F1D0E945F0F442091F041E01B
:101F9000B601601B710BC7018C0F9D1F0E945F0F64
:101FA00041E0B6016C1B7D0BC8018E0D9F1D0E9488
:101FB0005F0F332091F041E0B6016C0F7D1FC70128
:101FC000801B910B0E945F0F41E0B8016C0D7D1DDD
:101FD000C7018C1B9D0B0E945F0F222091F041E0F6
:101FE000B6016C1B7D0BC701801B910B0E945F0F1C
:101FF00041E0B601601B710BC7018C1B9D0B0E9459
:102000005F0FC017D10754F4B7FCA5CF01501109D9
:1020100082E0680E711CA60CB71C9DCFDF91CF919A
:102020001F910F91FF90EF90DF90CF90BF90AF90F6
:102030009F908F907F906F905F904F903F902F90E8
:1020400008952F923F924F925F926F927F928F925C
:102050009F92AF92BF92CF92DF92EF92FF920F9337
:102060001F93CF93DF93EC0141E06FE370E00E9498
:102070005F0F41E065E370E0CE010E945F0F41E039
:102080006AE370E0CE0105960E945F0F41E06AE3CB
:1020900070E0CE0105970E945F0F22242394312C1B
:1020A000F12CE12C05E010E036EF432E55245A9434
:1020B0004CEFC42EDD24DA948FEFE81AF80A82E0A0
:1020C000280E311CC20CD31C47018C0E9D1E41E012
:1020D00058018AE3A80EB11CB501C4010E945F0F2C
:1020E0003E016E187F0841E0B501C3010E945F0FF9
:1020F00041E08AE3A82EB12CA01AB10AB501C401AF
:102100000E945F0F41E0B501C3010E945F0F4701CC
:102110008AE3880E911C41E0B4015E01A00EB11E5D
:10212000C5010E945F0F41E0B4013E01601A710ACF
:10213000C3010E945F0F9AE3892E912C8E189F088D
:1021400041E0B401C5010E945F0F41E0B401C30149
:102150000E945F0FE016F1069CF0DF91CF911F9176
:102160000F91FF90EF90DF90CF90BF90AF909F9036
:102170008F907F906F905F904F903F902F90089539
:10218000D7FC9ACF0150110982E0480E511CC40CB3
:10219000D51C92CF8F929F92AF92BF92CF92DF9237
:1021A000EF92FF920F931F93CF93DF936D3089F0DF
:1021B000C0906602D09067026A30D1F41092650236
:1021C0001092640288E0C80ED11CD0926702C092BF
:1021D000660281E090E0DF91CF911F910F91FF9017
:1021E000EF90DF90CF90BF90AF909F908F90089529
:1021F0000091640210916502E5E06E9FE0011124F8
:10220000C45DDC4F4801F12CF5E0E12CFF1629F00C
:10221000CE010196FE01E490EC01B12CA12C4E2DD3
:102220004170B6016A0D7B1DC4010E945F0FE694E8
:10223000FFEFAF1ABF0A88E0A816B10481F7F39444
:10224000EFEF8E1A9E0AF6E0FF12DECF0A5F1F4FF5
:102250001093650200936402BCCFDF92EF92FF926D
:102260000F931F93CF93DF937C01D22E8B01040F2A
:10227000111DEB0177FF02C0D0E0C0E0C8010134BE
:10228000110514F080E490E0C817D9073CF44D2DF7
:10229000BE01C7010E945F0F2196F0CFDF91CF9161
:1022A0001F910F91FF90EF90DF9008952F923F9232
:1022B0004F925F926F927F928F929F92AF92BF9256
:1022C000CF92DF92EF92FF920F931F93CF93DF9302
:1022D00000D000D000D0CDB7DEB76C01762E542EE2
:1022E0004901602E98E0A92EB12C611103C089E04C
:1022F000A82EB12CCE0101967C018E010D5F1F4FDF
:102300009E012B5F3F4FA401652D872D0E94E4099C
:1023100009811A81552011F1B401990C880B990B90
:102320000E94083120E030E040E05FE30E94673126
:102330001B012C0120E030E0A9010E94423420E082
:1023400030E040E05FE387FD0CC0C201B1010E94B4
:10235000D6320E94B433C616D70644F48D809E80D0
:1023600009C0C201B1010E94D532F3CF8B809C809D
:10237000C61AD70ACA9CB001CB9C700DDA9C700DAE
:102380001124060F171FC40104976620B1F061E005
:1023900070E0711002C062E070E0060F171F6C0160
:1023A000C6012FEFC21AD20AC814D90491F020E056
:1023B00045E0B8010E942D11F3CF61E070E071108B
:1023C00002C062E070E0600F711F4BE55FE00E94A9
:1023D000DD0926960FB6F894DEBF0FBECDBFDF91A4
:1023E000CF911F910F91FF90EF90DF90CF90BF9012
:1023F000AF909F908F907F906F905F904F903F90A5
:102400002F9008950F93CF93DF93EC019E816A3054
:1024100059F48D818C836985960F9E8381E090E0CD
:10242000DF91CF910F910895262F61E0690F2A3334
:1024300098F4203378F5273249F140F4213261F1E4
:1024400098859C5F8C81890F8C83E8CF2C3231F189
:102450002E32B1F72FE309C0213490F32B35C0F0B1
:102460008FE9820F27548A3158F7062E000C770B1C
:102470008C81082E000C990B3F810AEF313009F056
:102480000BEF42E252E00E942208DACF21E4EDCFC6
:102490002154EBCF2C5FE9CF2EE3E7CF20E4E5CF4B
:1024A0000F93CF93DF93EC019E816A3059F48D81B5
:1024B0008C836985960F9E8381E090E0DF91CF91B8
:1024C0000F910895262F61E0690F2A3398F4203385
:1024D00078F5273249F140F4213261F198859D5F0A
:1024E0008C81890F8C83E8CF2C3231F12E32B1F7F9
:1024F0002FE309C0213490F32B35C0F08FE9820F10
:1025000027548A3158F7062E000C770B8C81082E41
:10251000000C990B3F810AEF313009F00BEF4AE5CF
:1025200051E00E942208DACF21E4EDCF2154EBCF15
:102530002C5FE9CF2EE3E7CF20E4E5CFECEAF2E031
:1025400084EC92E030E020E04191519161917191F1
:10255000240F351F8E179F07B9F78091790290914C
:102560007A02821B930B0895E091CC02F091CD0288
:102570003297E531F10508F034C0EF53FD4E0C946D
:10258000A434DC12F112D912DF12E212F112F112AC
:10259000D612E512F112F112F112F112F112F1124A
:1025A000EC12EC12F112D912F112D91282E090E081
:1025B000089581E090E0089583E090E0089584E03C
:1025C00090E0089585E090E0089580918B029091CD
:1025D0008C020397029728F48091890290918A02D5
:1025E000089590E080E00895CF93C82F84E00E9482
:1025F000460F811107C0CC23B1F088E00E94460F3E
:10260000882389F01092D2020E94B4129093D102D2
:102610008093D00280918B0290918C029093CD0296
:102620008093CC0281E0CF910895E4E8F7E08AE45A
:102630008583848387E3868369ED70E0CF010E9400
:10264000A60E8BE490E00E94211087E690E00C94A7
:102650002110CF92DF92EF92FF920F931F93CF93AF
:10266000DF9346E770E060E085E090E00E94EB07D2
:1026700046E76FE370E085E090E00E94EB0721E021
:1026800046E365E070E090E080E00E942D1121E0DB
:1026900046E365E070E08FE790E00E942D1141E095
:1026A00065E070E085E090E00E947D0F42E065E02B
:1026B00070E08AE790E00E947D0F44E06AE370E0FA
:1026C0008AE790E00E947D0F48E06AE370E085E0D1
:1026D00090E00E947D0F80918D02C2E4D7E08111CD
:1026E00022C00AE010E0F12CE12C8AE0C82ED12CA7
:1026F00080918E0290918F02E816F90684F58FEF93
:10270000E81AF80AD0926502C09264021093670238
:1027100000936602BE0188E997E00E94E60D065F1D
:102720001F4F2696E5CF1AE0F12CE12C0AE08091AC
:102730008E0290918F02E816F9068CF400939307AD
:102740000093920710939407BE018EE897E00E94D1
:10275000E60D8FEFE81AF80A175F2696E8CFDF91AB
:10276000CF911F910F91FF90EF90DF90CF90089540
:10277000BC01EEE8F7E096E0958394838CE08683D5
:10278000CF010C94E60D90E080E008958F929F9227
:10279000AF92BF92EF92FF920F931F93CF93DF936D
:1027A000CDB7DEB7A1970FB6F894DEBF0FBECDBF91
:1027B0007C01FA01CB0119A2223008F42AE08E0133
:1027C0000F5D1F4F822E912CB12CA12CBF01A501B2
:1027D00094010E94A432F901CA016A3074F5605D67
:1027E000D8016E938D01232B242B252B79F790E0B4
:1027F00080E0109789F0FD0101900020E9F7319702
:10280000AF014A1B5B0BD701ED91FC910280F38174
:10281000E02DB801C7010995A1960FB6F894DEBF67
:102820000FBECDBFDF91CF911F910F91FF90EF9021
:10283000BF90AF909F908F900895695CD1CFCF9259
:10284000DF92EF92FF920F931F93CF93DF9377FF67
:1028500021C06A017B01EC01E881F9810190F081DE
:10286000E02D6DE209958C0144275527BA014C19DA
:102870005D096E097F092AE0CE010E94C613800F10
:10288000911FDF91CF911F910F91FF90EF90DF90FB
:10289000CF9008952AE0DF91CF911F910F91FF9083
:1028A000EF90DF90CF900C94C613CF93DF93CFE1DE
:1028B000D0E020E04AE067E170E0CE010E942D11F7
:1028C0002196CF36D105A9F783E2809393078093B1
:1028D000920788E1809394074091750250917602A7
:1028E00060917702709178028EE897E0DF91CF9146
:1028F0000C941F14BC01EEE8F7E09AE095839483F2
:1029000088E18683CF010E94E60D48E566E170E02C
:102910008EE190E00E94EB0748E561E270E08EE115
:1029200090E00E94EB0721E04CE066E170E08EE170
:1029300090E00E942D1121E04CE066E170E085E717
:1029400090E00E942D110E94551442ED50E068E184
:1029500070E08FE690E00C94DD09CF92DF92EF9269
:10296000FF920F931F93CF93C82F8B0169017A01B8
:102970006E5F7F4F4BEC50E00E94DD09CA5FEEE8CE
:10298000F7E0C583C4830683B701A601CF01CF91C9
:102990001F910F91FF90EF90DF90CF900C941F1438
:1029A000CF93DF938091CC029091CD024197029713
:1029B00068F5C8E2D0E020E047E065E270E0CE01D3
:1029C0000E942D112196CF37D105A9F7E0918902F8
:1029D000F0918A02EE0FFF1FEE0FFF1FEC56FD4F26
:1029E000208131814281538160917502709176021C
:1029F00080917702909178020E9494349B01AC01FF
:102A000065E270E088E290E00E94AD14DF91CF9122
:102A10000C945514CF93DF93EC0188819981009732
:102A200011F00E944635198218821D821C821B8279
:102A30001A82DF91CF910895FC01808191810097E6
:102A400011F00C9446350895CF93C82F8091CA0297
:102A50009091CB0201969093CB028093CA02109280
:102A600074020E94383021EE3EE240E050E00E94C5
:102A70003B326058714C8F4F9F4F6093940270931C
:102A8000950280939602909397020E94383029E530
:102A90003BE140E050E00E943B3268577C4E8F4F54
:102AA0009F4F609398027093990280939A0290933B
:102AB0009B020E94383023E230E040E050E00E9468
:102AC0003B329B01AC01265F3F4F4F4F5F4FA4E667
:102AD000B0E00E945A3260939C0270939D028093F2
:102AE0009E0290939F020E9438302BE230E040E03B
:102AF00050E00E943B329B01AC012F5D3F4F4F4F96
:102B00005F4FAAE0B0E00E945A326093A002709337
:102B1000A1028093A2029093A3020E94383020E188
:102B200030E040E050E00E943B329B01AC01295F65
:102B30003F4F4F4F5F4FAAE0B0E00E945A32609380
:102B4000A4027093A5028093A6029093A7020E940C
:102B5000383025E030E040E050E00E943B329B01FD
:102B6000AC012F5F3F4F4F4F5F4FAAE0B0E00E9494
:102B70005A326093A8027093A9028093AA0290939C
:102B8000AB02CC23C1F160918102709182028091ED
:102B90008302909184020E9408312DEC3CEC4CE8B9
:102BA0005FE30E9467310E94EA330E94B43360936E
:102BB00081027093820280938302909384026091D9
:102BC0007D0270917E0280917F02909180020E942E
:102BD000083124E13EEA47E85FE30E9467310E9442
:102BE000EA330E94B43360937D0270937E02809337
:102BF0007F02909380021092D202CF9108950C949C
:102C000025320F931F93CF93DF938C01EB01FC01CF
:102C1000808191810097E1F068817981611571056A
:102C2000A9F0428153812C813D814217530770F0F6
:102C30000E9495368C819D81F801958384831D8245
:102C40001C82DF91CF911F910F9108950E9446350C
:102C500088819981F801918380838A819B81938304
:102C600082838C819D8195838483198218821B8243
:102C70001A82E5CF0F931F93CF93DF93EC018881E6
:102C80009981009759F02A813B812617370730F048
:102C900081E0DF91CF911F910F9108958B016F5FBC
:102CA0007F4F0E94CF35009759F0998388831B830B
:102CB0000A832C813D81232B59F7FC011082E8CF38
:102CC00080E0E7CFEF92FF920F931F93CF93DF93B4
:102CD000EC017B01CB010E9497300097A9F00C8199
:102CE0001D81080F191FB801CE010E943A168823D2
:102CF00061F0288139818C819D81B701820F931FFA
:102D00000E9490301D830C8381E0DF91CF911F9151
:102D10000F91FF90EF900895EF92FF920F931F9302
:102D2000CF93DF93FB01E080F180E114F10441F4E3
:102D300080E0DF91CF911F910F91FF90EF90089568
:102D40000481158101151105B1F0EC018C819D8183
:102D5000080F191FB801CE010E943A16882341F3CB
:102D6000288139818C819D81B701820F931F0E9438
:102D700095361D830C8381E0DCCFEF92FF920F9399
:102D80001F93CF93DF93EC018B016115710551F017
:102D9000CB010E9497307C01BC01CE010E943A1603
:102DA00081110BC0CE010E940A15CE01DF91CF9197
:102DB0001F910F91FF90EF900895FD82EC82B80172
:102DC000888199810E949030F0CFFC01118210829D
:102DD00013821282158214820C94BD16CF93DF9356
:102DE000EC016230710501F148F46115710581F063
:102DF00061307105B1F06FE271E00CC064307105B3
:102E0000C9F0A8F065307105B1F760E371E002C068
:102E10006EE471E0CE010E94E516CE01DF91CF9104
:102E2000089566E471E0F6CF61E471E0F3CF6CE3FE
:102E300071E0F0CF66E371E0EDCFCF93DF93EC016B
:102E40006230710501F148F46115710581F061305E
:102E50007105B1F065EE70E00CC064307105C9F029
:102E6000A8F065307105B1F766EE70E002C062E26D
:102E700071E0CE010E94E516CE01DF91CF91089559
:102E800065E171E0F6CF6BE071E0F3CF6EEF70E0DB
:102E9000F0CF63EF70E0EDCFEF92FF920F931F93AF
:102EA000CF93DF93EC017B018A01BA010E943A16AD
:102EB00081110BC0CE010E940A15CE01DF91CF9186
:102EC0001F910F91FF90EF9008951D830C83B70120
:102ED000888199810E949536F0CFFB0101900020F6
:102EE000E9F73197AF01461B570B0C944C170F9322
:102EF0001F93CF93DF93CDB7DEB762970FB6F894E9
:102F0000DEBF0FBECDBF8C01CB01F8011182108254
:102F100013821282158214824AE0BE016F5F7F4FD6
:102F20000E94A030BE016F5F7F4FC8010E946D17E5
:102F300062960FB6F894DEBF0FBECDBFDF91CF9182
:102F40001F910F9108950F931F93CF93DF93CDB7E8
:102F5000DEB7A2970FB6F894DEBF0FBECDBF8C01CF
:102F6000CB01BA01F80111821082138212821582FC
:102F700014822AE0AE014F5F5F4F0E94AB30BE016A
:102F80006F5F7F4FC8010E946D17A2960FB6F8942D
:102F9000DEBF0FBECDBFDF91CF911F910F9108957E
:102FA0002F923F924F925F926F927F928F929F9259
:102FB000AF92BF92CF92DF92EF92FF920F931F9347
:102FC000CF93DF93CDB7DEB762970FB6F894DEBF2D
:102FD0000FBECDBF2C019E012F5F3F4F490139012C
:102FE0001C01D12CC12C10E000E0B12CA12CF1016E
:102FF00041915191619171911F01CE010D960E94F5
:10300000A317E988FA88CE010D960E941C15B60117
:10301000CE010D960E94EE1689899A89E80EF91E56
:10302000FFEFEF1AFF0AF301E192F1923F01CE01A7
:103030000D960E941C15F3E0CF16D1040CF03FC092
:10304000AE14BF040CF457012FEFC21AD20A36E0B7
:10305000C316D10461F680E6C82E87E0D82EF12C85
:10306000E12C150183E0E816F1040CF01801B7011A
:10307000CE010D960E94EE16BE01635F7F4FC60122
:103080000E940116CE010D960E941C1568E571E0A4
:10309000C6010E946216712C612CF401808191811D
:1030A0009101281B390B6216730674F466E571E012
:1030B000C6010E9462163FEF631A730AEECF0E1527
:1030C0001F0514F68701C0CFF20141915191619122
:1030D00071912F01CE010D960E94A317BE01635F6F
:1030E0007F4FC6010E948C16CE010D960E941C15C2
:1030F000FFEFEF1AFF0A26E0C20ED11C32E0830E6A
:10310000911C86E0E816F10409F0ABCFF092C902F9
:10311000E092C80281E08093C6020A0D1B1D0731B0
:1031200011050CF480E08093C70262960FB6F89404
:10313000DEBF0FBECDBFDF91CF911F910F91FF90EA
:10314000EF90DF90CF90BF90AF909F908F907F9047
:103150006F905F904F903F902F900895EF92FF9265
:103160000F931F93CF93DF9300D000D000D0CDB743
:10317000DEB78C019CE3E92EF12C20E04CE069E005
:1031800070E0C7010E942D118FEFE81AF80A80E85D
:10319000E816F10491F7000F111F000F111FF8013D
:1031A000E455FD4F4081518162817381CE010196CA
:1031B0000E94A3178D818195880F880F845A809370
:1031C0008907809388078DE080938A0748E050E064
:1031D00064E571E084E897E00E94CA0EBE016F5F6B
:1031E0007F4F84E897E00E94E60DCE0101960E9491
:1031F0001C1526960FB6F894DEBF0FBECDBFDF912B
:10320000CF911F910F91FF90EF900895EF92FF9251
:103210000F931F93CF93DF9300D000D000D0CDB792
:10322000DEB78091CC029091CD02099709F05EC083
:103230000E949E128C01BC01CE0101960E9477175C
:10324000ED80FE80CE0101960E941C1581E08093E6
:1032500089078093880710928A0764EC70E084E8FD
:1032600097E00E94A60E40917B0250917C02052EB1
:10327000000C660B770B84E897E00E941F1487E12F
:1032800090E08E199F09880F991F880F991F8093CE
:1032900089078093880710928A076AEB70E084E8B8
:1032A00097E00E94A60EA801110F660B770B84E829
:1032B00097E00E941F1410E000E021E041E068E088
:1032C00070E0C8010E942D110F5F1F4F00381105DB
:1032D000A1F726960FB6F894DEBF0FBECDBFDF91E3
:1032E000CF911F910F91FF90EF900895409185022B
:1032F000509186026091870270918802CE010196FA
:103300000E94A317ED80FE80CE0101960E941C153D
:1033100000E210E00E191F09000F111F000F111F0E
:103320008091CC029091CD029C0125503109223030
:10333000310508F052C021E02093890720938807C7
:1033400010928A0760EB70E0059711F465EB70E06E
:1033500084E897E00E94A60E4BEC50E061E070E03C
:1033600083E190E00E94DD0989E1809389078093E1
:10337000880710928A078091CC029091CD02059720
:1033800019F54091810250918202609183027091FF
:10339000840284E897E00E941F144BEC50E061E047
:1033A00070E0C80106970E94DD0900938907009329
:1033B000880710928A074091850250918602609199
:1033C00087027091880273CF40917D0250917E02F6
:1033D00060917F0270918002DCCF81E08093890749
:1033E0008093880710928A076CEA70E084E897E07F
:1033F0000E94A60E8EE08093890780938807109222
:103400008A074091CA025091CB02052E000C660B30
:10341000770BBFCF1F920F920FB60F9211248F938D
:103420009F938091E1009091E100937F9093E10060
:1034300083FF0FC01092E90091E09093EB0010928F
:10344000EC0092E39093ED001092F10298E09093DB
:10345000F00082FF22C093E09093E9009091F20087
:10346000992319F09AE39093E8009091E20299234E
:1034700041F09091E20291509093E202911101C0CB
:103480005D9A9091F002992341F09091F002915051
:103490009093F002911101C0289A84FF18C0809186
:1034A000E2008E7E81608093E2008091E1008F7E59
:1034B0008093E1008091E3028E7E80618093E3023D
:1034C0009F918F910F900FBE0F901F90189580FFC6
:1034D000F7CF8091E2008E7E80618093E200809140
:1034E000E1008E7E8093E1008091E3028E7E816018
:1034F000E5CF1F920F920FB60F921124CF92DF9259
:10350000EF92FF920F931F932F933F934F935F93ED
:103510006F937F938F939F93AF93BF93EF93FF939B
:10352000CF93DF93CDB7DEB76C97DEBFCDBF1092E0
:10353000E9008091E80083FF25C068E0CE01459650
:103540000E94FB0C82EF8093E8008D8987FF39C0D1
:103550009091E80090FFFCCF982F907609F034C14D
:103560009E894F89588D2F89F88C911131C08038F0
:1035700061F58091E1028093F1001092F1008EEFED
:103580008093E8006C960FB6F894DEBF0FBECDBFF7
:10359000DF91CF91FF91EF91BF91AF919F918F916B
:1035A0007F916F915F914F913F912F911F910F915B
:1035B000FF90EF90DF90CF900F900FBE0F901F9075
:1035C00018959EEF9093E800C7CF1092F100D5CFE9
:1035D000913059F48111D3CF4130510581F680915A
:1035E000E1028D7F8093E102CACF933049F48111CB
:1035F000C6CF4130510519F68091E1028260F2CFC9
:10360000953041F48091E80080FFFCCF2068209342
:10361000E300B5CF963009F0A9C00B8D1C8D22E0D8
:103620001092E9001092DF021092DE02F2122EC018
:103630001092DD021092DC020E94CA0C1F8299E0F7
:103640009983FA8291E09E8390EA98879AEF99870E
:103650002091DE023091DF02275F3F4F3C832B83B6
:103660008D831092E9001092DF021092DE02109317
:10367000DD020093DC0249E050E0BE016F5F7F4F46
:1036800080E00E94A40C0E94CA0C79CF1093DD0246
:103690000093DC020E94E10BDC0112960D911C915B
:1036A0000115110509F451C1D801ED91FC91048077
:1036B000F581E02DBE016B5E7F4FC8010995009733
:1036C00009F03EC1F80100851185EACFF3E0FF1251
:1036D0000EC08F89882309F440C0823061F440E82D
:1036E00060E18AE49FE00E94F51C811148CF81E2ED
:1036F0008093EB0047CF813029F440E86BE08EE304
:103700009FE0F1CF833099F70E94E10BDC01129624
:10371000ED90FC908E010F5F1F4F6801E114F104E2
:1037200079F0D701ED91FC910680F781E02DB80189
:10373000C7010995080F111DF701E084F184EECF50
:10374000D8011C92F60101900020E9F73197BF01E2
:103750006C197D0940E0C601C6CF68E27FE0FB013D
:10376000449150E080E80E94A40C09CF973009F4FE
:10377000BECF983021F481E08093F10000CF9930E2
:1037800009F0FDCE837009F0B2CFE8E1F1E081E00D
:1037900031E096E32191222371F08093E900309388
:1037A000EB00DF0111972C912093EC009093ED003A
:1037B0008F5F873079F78EE78093EA001092EA00F6
:1037C0008F898093F102DBCE8B8D9C8D1092E90066
:1037D0001092DF021092DE029093DD028093DC02F1
:1037E000898D811192C08E899D89913A49F48132E7
:1037F00009F07DCF47E050E065E071E080E0B3CFB5
:10380000913209F074CF833269F48F89988DB0E0DA
:10381000A0E08093010190930201A0930301B09373
:103820000401ADCE803269F48091E80082FFFCCFC4
:1038300067E085E091E00E94FB0C8BEF8093E8004D
:103840009ECE823209F09BCE8F8980930C01EEEFE1
:10385000FFE7859194918B3F9C4D51F1E0E0F8E0BA
:103860008091050190910601A0910701B091080196
:10387000803B9440A105B105F1F480910C0180FDDD
:103880001AC0EE3F8AE0F80789F587E797E791834A
:103890008083809160008093E00288E19BE00FB616
:1038A000F894A895809360000FBE9093600067CE57
:1038B000EEEFFAE0D5CF808191818737974709F005
:1038C0005ECEA895809160008861809360008091B1
:1038D000E00280936000EE3F2AE0F20789F08091D9
:1038E000FE0A9091FF0A9183808349CE8081918165
:1038F0008737980751F29093FF0A8093FE0AC5CF4D
:103900001092FF0A1092FE0A3ACE0E94E10BDC01EF
:1039100012960D911C910115110509F4E8CED801FC
:10392000ED91FC910190F081E02DBE016B5E7F4F27
:10393000C8010995811123CEF80100851185EBCFCF
:10394000181619060CF41BCED2CEF1E0FF12BECE33
:103950006CE27FE004CF1F920F920FB60F921124FA
:103960002F933F938F939F93AF93BF938091D402F4
:103970009091D502A091D602B091D7023091D30296
:1039800023E0230F2D3758F50196A11DB11D20937B
:10399000D3028093D4029093D502A093D602B09321
:1039A000D7028091D8029091D902A091DA02B09109
:1039B000DB020196A11DB11D8093D8029093D9021C
:1039C000A093DA02B093DB02BF91AF919F918F91E8
:1039D0003F912F910F900FBE0F901F90189526E8E2
:1039E000230F0296A11DB11DD2CFEF92FF920F932C
:1039F0001F93CF93DF93F82E192FE62E042F81E02B
:103A0000860F880F0E94760C83E00E94760CCF2DE3
:103A1000D12FEC0EFD2EF11CCE15DF05B9F007FFFE
:103A200013C0FE0184910E94760C182F80E00E9442
:103A3000760C812321968111EFCFDF91CF911F91D9
:103A40000F91FF90EF9008958881EDCF81E0F5CF41
:103A5000CF93DF931092F5061092F40688EE93E070
:103A6000A0E0B0E08093F6069093F706A093F806E6
:103A7000B093F90682E291E09093F3068093F20608
:103A80008FEF9FEF9093FF068093FE0610929B07A7
:103A900010929A078CE491E090939907809398078D
:103AA000109291071092900780E491E090938F0715
:103AB00080938E0798E09093970781E08093960714
:103AC0001092930710929407109292078093950793
:103AD000109287071092860724E331E03093850720
:103AE0002093840790938D0780938C071092890709
:103AF00010928A071092880780938B07C0E6D7E060
:103B0000198218821B821A821D821C8250E040E0BA
:103B100067EF71E0CE010E944C17269687E0C4380B
:103B2000D80771F7C2E4D7E0198218821B821A8283
:103B30001D821C8250E040E067EF71E0CE010E94E0
:103B40004C17269687E0C036D80771F7DF91CF91E2
:103B50000895CF93DF93CDB7DEB72E970FB6F894C5
:103B6000DEBF0FBECDBF789484B5826084BD84B5BE
:103B7000816084BD85B5826085BD85B5816085BD68
:103B800080916E00816080936E0010928100809120
:103B900081008260809381008091810081608093A8
:103BA00081008091800081608093800080919100ED
:103BB0008260809391008091910081608093910058
:103BC000809190008160809390008091C10084601A
:103BD0008093C1008091C10082608093C100809178
:103BE000C10081608093C1008091C3008160809397
:103BF000C3008091C00082608093C0008091C200A9
:103C000081608093C20080917A00846080937A0002
:103C100080917A00826080937A0080917A0081603E
:103C200080937A0080917A00806880937A00109265
:103C3000F1021092E1021092E3028091D7008160BC
:103C40008093D70080EA8093D80089B5806189BDD0
:103C500089B5826089BD09B400FEFDCF61E070E0E6
:103C600080E090E00E942D0D8091D8008F7C8061D3
:103C70008093D8008091E000807F8093E000809165
:103C8000E1008E7E8093E1008DE08093E200559A02
:103C9000209A0E94060F82E48093000180916400C4
:103CA0008E7F8093640080917A00806480937A0094
:103CB00080917A0086FDFCCF009178001091790008
:103CC0000E94080DAB01BC01C801B0E0A0E0DC011E
:103CD000992788276C017D01C40ED51EE61EF71EAC
:103CE000C701B60120916400216020936400611532
:103CF00071058105910511F00E9487301092CD0267
:103D00001092CC021092D2020E94060F0E945C0F09
:103D100080E80E94510F8823A9F05C9885EA8EBD47
:103D200000000DB407FEFDCF5C9A2E982F982D98B9
:103D30008091640080628093640081E083BF8895F5
:103D400013BEFCCF84E00E94510F882309F448C0C1
:103D50002D9884E80E94510F8823E1F00E94F70E0D
:103D600088EC90E00E94F90E2F9882E090E00E948B
:103D700025328F3F29F06FEF82E090E00E942D32D4
:103D800084EF91E00E94F90E2F9A84E80E94510F6F
:103D90008111FBCF84E10E94510F8823E1F00E9442
:103DA000F70E88EC90E00E94F90E2E9882E090E0E9
:103DB0000E942532882329F060E082E090E00E9492
:103DC0002D3284EF91E00E94F90E2E9A84E10E9438
:103DD000510F8111FBCF88EC90E00E94F90EB2CF19
:103DE0000E94F70E82E090E00E94FF158823E1F127
:103DF0003E9A3F9A81E090E00E94FF1581FF13C038
:103E0000082F0470302E82FD2E9801EF1FEFA8E0DE
:103E1000AA2EB12C80E40E94510F882341F12E9AE2
:103E20002F9A0E94F70E82E390E00E94F90E0E9402
:103E3000FE0E8111F8CF8FB7F8944091D4025091C3
:103E4000D5026091D6027091D7028FBF8091620235
:103E5000882309F4D0C01092620280E090E0892BA0
:103E600051F30E940000E7CF3E983F98C3CF332024
:103E700029F00430110511F42E9A2F9881E00E9448
:103E8000DC07980117FF04C022273327201B310BC2
:103E900027703327C80117FD0796F3E0959587959E
:103EA000FA95E1F717FF05C00197A501421B530BD7
:103EB0009A01AC015695542F4427579547954E507B
:103EC0005D4FF12CE12C2501421A530A8E3F6FEF12
:103ED000960709F43EC0DA0170E060E0F701E75CA4
:103EE000F74F4F013A01F0E86F0E711C8F3F9807B2
:103EF00081F0F401E60FF71FE491022E01C0EE0FEE
:103F00000A94EAF75496FC915497EF2B5496EC934D
:103F1000549721153105B9F0F401E60FF71F2490ED
:103F20006301C60ED71EE22DF0E0042C02C0F59509
:103F3000E7950A94E2F7FE87ED87F6012488FD8570
:103F40002F2AF601248A6F5F7F4F1196683571051D
:103F500069F60196F8E5EF0EF11C40585F4F60EBF3
:103F6000E616F10409F0B2CF0E945C0F8FE090E0FA
:103F70000E94F90E0F5F1F4F0931110509F04ACF5A
:103F8000332011F02F9A2D9880E991E00E94F90ECC
:103F90000E94F70E81E090E00E94FF1580FF43CF62
:103FA0008AE090E00E94FF159FEF980F9E3F08F077
:103FB0003ACF22E330E0309365022093640228E395
:103FC00030E030936702209366020BE010E0682F28
:103FD00088E997E00E94CA10C8010E94FF150F5F90
:103FE0001F4F0131110599F70E945C0F88EE93E095
:103FF0000E94F90E18CF80916302942F981B892F8D
:1040000090910001891748F48F5F891708F025CF38
:1040100081E083BF889513BE20CF81E08093620248
:1040200040936302809160029091610201969093A7
:1040300061028093600280916902809368020E940D
:10404000FE0E809369028091D2028111FDC0209101
:10405000CC023091CD02E2EFF2E081118FEF00242B
:1040600081938193819381930394D1F71092670296
:104070001092660210926502109264028091D00242
:104080009091D1029093CF028093CE021092D102F0
:104090001092D0022130310561F48091CA029091D2
:1040A000CB024F9734F087E190E09093CD0280935C
:1040B000CC028091CC029091CD028831910508F01C
:1040C000C5C4FC01EA59FF4D0C94A4347E20C220E3
:1040D000A6216C216C2122224B226422C9224D216F
:1040E000562356235623562362238E232B23AD2398
:1040F000AD235024502450245024BD244CE65EE0CF
:1041000070E060E090E080E00E94DD094CE65EE057
:1041100070E060E082E690E00E94DD098AE290E0D3
:1041200090936502809364028FE090E09093670221
:104130008093660263E67EE088E997E00E94A60E1F
:1041400087E680938907809388078AE380938A07AC
:104150006CE57EE084E897E00E94A60E6AE47EE0CB
:1041600080E697E00E94BD1681E090E09093C9023E
:104170008093C8021092C7021092C60241E050E03C
:1041800060E04DC00E9406196091C4027091C502A2
:10419000CE0101960E941D17CE0101960E94B81310
:1041A000CE0101960E941C1560E47EE080E697E057
:1041B0000E94BD1665E37EE086E697E00E94BD168C
:1041C0006AE27EE08CE697E00E94BD1666E27EE041
:1041D00082E797E00E94BD168091C4029091C502CB
:1041E000892B09F057C06BE17EE088E797E00E94D9
:1041F000BD1666E17EE08EE797E00E94BD1686E080
:1042000090E09093C9028093C8021092C70281E0A7
:104210008093C6024091C8025091C90261E080E0DB
:104220000E94F40D2091C8023091C90200E0409133
:10423000C6026091C7028091CE029091CF020E9487
:10424000561181E08093D202C090CC02D090CD0272
:10425000B8E1CB16D10408F09AC4F601EE5CFE4D2D
:104260000C94A43443254325432543254325432566
:1042700043252B2C9F2B9F2B9F2BA32BA32BA32BB7
:104280009F2B9F2BA32B242D242D242D242D242D37
:10429000242D9F2B84E090E0B4CF0E9406196BE0A0
:1042A0007EE0CE0101960E94E516CE0101960E94A5
:1042B000B813CE0101960E941C158CEA92E00E9470
:1042C000D0174091C8025091C9026091C6028091F6
:1042D000C7020E94F40DB5CF0E9406198091CC024E
:1042E0009091CD0261E07EE0039711F066EF7DE0F2
:1042F000CE0101960E94E516CE0101960E94B813E8
:10430000CE0101960E941C1584E992E00E94D0170C
:104310004091C8025091C9026091C6028091C702C3
:104320000E94F40DE090CE02F090CF022091C802DE
:104330003091C90200E04091C6026091C702C701F6
:104340000E945611C7010E94AE187BCF0E94061929
:104350006CEE7DE0CE0107960E94E5166091C402E6
:104360007091C502CE0101960E941D17BE016F5FBC
:104370007F4FCE0107960E948C16CE0101960E94B7
:104380001C151A8219821C821B821E821D826F815B
:1043900078856115710531F04B855C85CE010196FC
:1043A0000E944C17CE0101960E94B813CE010196CF
:1043B0000E941C1570E6E72E77E0F72E70E060E0B3
:1043C0008B010F5F1F4F8091C4029091C502681747
:1043D00079070CF0B801CE0101960E941D17BE01AD
:1043E0006F5F7F4FC7010E940116CE0101960E94A8
:1043F0001C15A6E0EA0EF11CB8010530110501F705
:104400001093C9020093C80281E08093C702809391
:10441000C60245E050E061E00E94F40D2091C80220
:104420003091C90200E04091C6026091C7028091BC
:10443000CE029091CF020E945611CE0107960E94A3
:104440001C15FFCE0E94061961EE7DE0CE0101969B
:104450000E94E516CE0101960E94B813CE01019686
:104460000E941C1566ED7DE080E697E00E94BD1677
:1044700069EC7DE086E697E00E94BD1682E090E060
:104480009093C9028093C8021092C7021092C6028C
:1044900042E050E075CE0E94061964EC7DE0CE014A
:1044A00001960E94E516CE0101960E94B813CE0136
:1044B00001960E941C1566EB7DE080E697E00E9465
:1044C000BD1667EA7DE0D6CF68E97DE082E497E03B
:1044D0000E94BD166DE87DE088E497E00E94BD165D
:1044E0006091920270919302CE0101960E9477171B
:1044F000BE016F5F7F4F88E497E00E948C16CE016B
:1045000001960E941C1567E87DE088E497E00E9410
:10451000621666E77DE08EE497E00E94BD1668E6CD
:104520007DE084E597E00E94BD1660919002709155
:104530009102CE0101960E947717BE016F5F7F4FF7
:1045400084E597E00E948C16CE0101960E941C150E
:1045500084E090E090938F0280938E0210928D02FF
:104560000E94291382E4809389078093880787E358
:1045700080938A076FE97CE084E897E00E94A60EAA
:1045800083E490E00E94211087E690E00E942110D1
:1045900058CE0E9438306B017C016FE87CE082E4E9
:1045A00097E00E94BD1668E87CE088E497E00E94EE
:1045B000BD1687E090E090938C0280938B0283E09D
:1045C00090E090938F0280938E0210928D02C7012B
:1045D000B60122E030E040E050E00E943B32672B21
:1045E00079F463E87CE088E497E00E9462166AE769
:1045F0007CE08EE497E00E94BD160E94291321CE34
:1046000063E77CE088E497E00E94621669E67CE05C
:104610008EE497E00E94BD168091900290919102E5
:1046200003979093910280939002181619062CF329
:1046300069E57CE084E597E00E94BD1684E090E0A7
:1046400090938F0280938E0287E190E090938C028A
:1046500080938B02D2CF66E57DE082E497E00E94F2
:10466000BD1668E47DE088E497E00E94BD1669E32A
:104670007DE08EE497E00E94BD166DE27DE084E56A
:1046800097E00E94BD1684E090E090938F028093A3
:104690008E0210928D020E9429130E94151381E050
:1046A00090E090938C0280938B02CBCD0E942913D3
:1046B0008091CC029091CD020A9709F4C2CD0E945C
:1046C0001513BFCD6DE571E082E497E00E946D1790
:1046D00060E771E088E497E00E946D1765E871E09B
:1046E0008EE497E00E946D1769E971E084E597E038
:1046F0000E946D176BEA71E08AE597E00E946D17E2
:1047000085E090E090938F0280938E0281E0809309
:104710008D020E9429138FE090E0C3CF67EF71E014
:1047200082E497E00E946D176FEB71E088E497E0F8
:104730000E946D176EEC71E08EE497E00E946D1799
:1047400083E090E090938F0280938E0210928D020E
:104750000E94291387E190E0A4CF66E27DE04197B3
:1047600011F060E27DE082E497E00E94BD16609166
:10477000890270918A02CE0101960E94EE16BE0156
:104780006F5F7F4F82E497E00E948C16CE01019606
:104790000E941C156CE27DE088E497E00E94BD1643
:1047A0006BE27DE08EE497E00E94BD168091CC0222
:1047B0009091CD0261E17DE0419711F06BE07DE0E9
:1047C00084E597E00E94BD1667E17DE08AE597E009
:1047D0000E94BD1685E090E090938F0280938E0238
:1047E00081E080938D020E942913E0918902F0916B
:1047F0008A02EE0FFF1FEE0FFF1FEC56FD4F2081C8
:104800003181428153816091460770914707E5E00D
:10481000E69FC001E79F900D11246AE070E00F96BB
:104820000E94AD148091CC029091CD024197E9F4A1
:104830002091850230918602409187025091880232
:104840006EE270E087E390E00E94AD140E94D01405
:1048500067E07DE0CE0101960E94E516CE0101964B
:104860000E947A14CE010196EACD87E380939307E4
:10487000809392078EE280939407E0918902F091F1
:104880008A02EE0FFF1FEE0FFF1FE455FD4F408120
:104890005181628173818EE897E00E941F14D6CF08
:1048A0006CEF7CE08331910559F06FEE7CE0843150
:1048B000910531F061EE7CE0459711F062ED7CE00E
:1048C00082E497E00E94BD1666E07DE088E497E010
:1048D0000E94BD1665E07DE08EE497E00E94BD1663
:1048E00080918B0290918C0261EC7CE0059711F035
:1048F00069EB7CE084E597E00E94BD1669EC7CE002
:104900008AE597E00E94BD1685E090E090938F02C3
:1049100080938E0281E080938D020E942913809102
:104920008B0290918C020597F9F4209181023091CD
:104930008202409183025091840265E270E082E33A
:1049400090E00E94AD142091850230918602409142
:104950008702509188026EE270E087E390E00E9447
:10496000AD1465EB7CE076CF20917D0230917E0224
:1049700040917F0250918002E0CF60917D02709162
:104980007E0280917F0290918002009185021091B9
:1049900086022091870230918802600F711F821F6A
:1049A000931F009181021091820220918302309125
:1049B0008402601B710B820B930B0E94083120E074
:1049C00030E04CEF51E40E9442330E944D340E948B
:1049D000EA330E94B4336B0167EF71E082E497E041
:1049E0000E946D176CED71E088E497E00E946D17EE
:1049F00069EE71E08EE497E00E946D17B6016536AE
:104A0000710514F064E670E0CE0101960E947717FC
:104A1000BE016F5F7F4F8EE497E00E948C16CE013F
:104A200001960E941C1568EF71E084E597E00E94F2
:104A30006D1710928D0284E090E090938F02809326
:104A40008E0210928C0210928B02D7CD85E090E0FE
:104A5000909365028093640290936702809366024C
:104A60006EEA7CE088E997E00E94A60E4091CC02B5
:104A70005091CD02052E000C660B770B88E997E06C
:104A80000E941F14DECB80E80E94460F81111AC0DD
:104A900080E10E94460F811115C080E20E94460FFE
:104AA000811110C080E40E94460F81110BC088E084
:104AB0000E94460F811106C084E00E94460F8823A1
:104AC00009F465C0A090C802B090C9027090C602F7
:104AD000E090CE02F090CF0201E09501472D609169
:104AE000C702C7010E945611B5010B2C000C880BA0
:104AF000990B0E94083120E030E040E05FE30E9423
:104B000067311B012C0120E030E0A9010E944234F2
:104B100020E030E040E05FE387FD3CC0C201B1012E
:104B20000E94D6320E94B4338B0188248394912C46
:104B3000E616F7061CF032E0832E912C80E10E94ED
:104B4000460F8823A1F1EFEFEE1AFE0AEA14FB04E8
:104B500034F5F092CF02E092CE02E090CE02F090D7
:104B6000CF022091C8023091C90200E04091C602F4
:104B70006091C702C7010E9456118091CC029091AA
:104B8000CD020397029718F4C7010E94AE180E9445
:104B90005C0F63C9C201B1010E94D532C3CFF1E0FD
:104BA000AF1AB108B092CF02A092CE02D6CF80E861
:104BB0000E94460F882371F001E0E01AF108F0929C
:104BC000CF02E092CE02F7FEC8CF1092CF02109231
:104BD000CE02C3CF80E40E94460F8823D9F077200D
:104BE000A9F08A94892891F4E00EF11EF092CF0288
:104BF000E092CE028091CE029091CF028A159B0561
:104C00000CF4ABCF41E0A41AB108CCCF3FEFE31ACC
:104C1000F30AECCF80E20E94460F8823B9F0772098
:104C200089F052E08516910469F4E01AF10AF092D5
:104C3000CF02E092CE028091CE029091CF0297FFF8
:104C40008CCFC3CF61E0E61AF108F1CF88E00E9473
:104C5000460F882309F45AC51092D20283E0C81681
:104C6000D10409F4BEC308F05AC0A1E0CA16D104A9
:104C700009F486C0B2E0CB16D10409F4B0C0EF2825
:104C800009F06BCF81E090E09093CD028093CC024D
:104C900020ED37E040E050E020938502309386021B
:104CA000409387025093880288E893E1A0E0B0E047
:104CB0008093810290938202A0938302B093840236
:104CC00010927D0210927E0210927F02109280025A
:104CD0001092C5021092C40210927C0210927B02C4
:104CE00084E690E090937A028093790282E390E0E8
:104CF0009093910280939002ECEAF2E084EC92E0CF
:104D000011921192119211928E179F07C9F710926A
:104D1000CB021092CA0280E00E9424151ECFE5E06B
:104D2000CE16D10409F47DC408F422C406E0C016EE
:104D3000D10409F0A4CF86E090E090938C02809398
:104D40008B021092750210927602109277021092E6
:104D50007802E114F10409F4CAC4EA94EF2809F0D6
:104D6000FCCE86E190E09093CD028093CC028091BE
:104D70007D0290917E02A0917F02B091800220C4BA
:104D8000D0928C02C0928B0292E0E916F104F1F00D
:104D900074F4E114F104B9F084E090E0EA94EF28AF
:104DA00009F0DBCE9093CD028093CC02D6CEE4E026
:104DB000EE16F10489F06CF086E090E005E0E01674
:104DC000F10481F3CACE83E090E0ECCF89E090E07B
:104DD000E9CF82E090E0E6CF85E090E0E3CF8091FC
:104DE000C4029091C502E816F9061CF01FEFE11A03
:104DF000F10AF092C502E092C40281E00E942415FB
:104E00000E94383024E130E040E050E00E943B3224
:104E10009B0141E050E050938C0240938B02109232
:104E20008D02FB013197E131F10508F0D5C2E55E55
:104E3000F84D0C94A4342C2753277227A527A527B7
:104E4000D027D027FD27442844284428A528A52872
:104E5000F9281A294929B92963ED7BE082E497E012
:104E60000E94BD1661EC7BE088E497E00E94BD16CD
:104E700068EB7BE08EE497E00E94BD1683E090E053
:104E800090938F0280938E0222E030E040E050E069
:104E90002093A8023093A9024093AA025093AB0238
:104EA0008AE090E07FCF67EA7BE082E497E00E94AF
:104EB000BD1667E97BE088E497E00E94BD1682E0BA
:104EC00090E090938F0280938E028AE790E0A0E0BA
:104ED000B0E08093A0029093A102A093A202B093AD
:104EE000A302DECF66E87BE082E497E00E94BD1675
:104EF00068E77BE088E497E00E94BD1667E67BE008
:104F00008EE497E00E94BD166AE57BE084E597E0B9
:104F10000E94BD1684E090E090938F0280938E02F1
:104F20000E9438302EE734E040E050E00E943B32EF
:104F30006E5A7C4F8F4F9F4F6093980270939902E7
:104F400080939A0290939B02ABCF6AE47BE082E469
:104F500097E00E94BD166BE37BE088E497E00E9437
:104F6000BD166DE27BE08EE497E00E94BD1663E221
:104F70007BE084E597E00E94BD1684E090E090938A
:104F80008F0280938E020E94383029EA31E640E099
:104F900050E00E943B32605B794B8F4F9F4FCCCFEC
:104FA00064E17BE082E497E00E94BD1663E07BE071
:104FB00088E497E00E94BD1660EF7AE08EE497E007
:104FC0000E94BD1683E090E090938F0280938E0242
:104FD0000E94383021E63AEE40E050E00E943B3239
:104FE0006058774C8E4F9F4F609394027093950258
:104FF000809396029093970253CF61EE7AE082E419
:1050000097E00E94BD1665ED7AE088E497E00E9483
:10501000BD1682E090E090938F0280938E026091A3
:1050200085027091860280918702909188020E9489
:10503000083120E030E040E450E40E9442336B014C
:105040007C0120E030E0A9010E94423420E030E001
:1050500040E05FE387FD13C0C701B6010E94D6326E
:105060000E94B433660F771F881F991F60938502D3
:1050700070938602809387029093880211CFC701B4
:10508000B6010E94D532ECCFECEAF2E090E080E08D
:105090004191519161917191840F951F42E0E43CDF
:1050A000F407B1F7C2970CF447C382E090E02930CF
:1050B000310539F084E090E02A30310511F085E0C7
:1050C00090E0909393028093920269EC7AE082E4FC
:1050D00097E00E94BD1664EC7AE088E497E00E94B5
:1050E000BD16609192027091930261507109CE01D8
:1050F00001960E947717BE016F5F7F4F88E497E0AB
:105100000E948C16CE0101960E941C156CEB7AE071
:1051100088E497E00E94621660EB7AE08EE497E004
:105120000E94BD1665EA7AE084E597E00E94BD160C
:1051300084E090E090938F0280938E0287E090E06D
:1051400090938C0280938B02ABCE809185029091DC
:105150008602A0918702B0918802843F9140A10508
:10516000B1050CF4E9C20E949E1205970CF4E4C24A
:105170000E94383023E030E040E050E00E943B32B3
:105180006B0166E97AE082E497E00E94BD1662E076
:10519000C616D104C8F469E77AE0CD2811F069E6B3
:1051A0007AE088E497E00E94BD1669E87AE08EE430
:1051B00097E00E94BD1683E090E090938F02809369
:1051C0008E028BE090E0EECD6BE57AE088E497E02C
:1051D0000E94BD166DE47AE08EE497E00E94BD1651
:1051E00064E47AE084E597E00E94BD1684E090E0F4
:1051F000E4CF63E37AE082E497E00E94BD1663E2C5
:105200007AE088E497E00E94BD1661E17AE08EE4DE
:1052100097E00E94BD1660E07AE084E597E00E9486
:10522000BD1684E090E090938F0280938E028DE013
:1052300090E0B8CD8091850290918602A09187027E
:10524000B09188028C329140A105B1050CF474C272
:105250006DEE79E082E497E00E94BD166DED79E095
:1052600088E497E00E94BD166EEC79E08EE497E04A
:105270000E94BD1663EC79E084E597E00E94BD16BC
:1052800084E090E090938F0280938E028CE090E017
:1052900089CD0E949E1208970CF44EC20E943830AD
:1052A00027E030E040E050E00E943B328B010F5F8E
:1052B0001F4F0E94383026E030E040E050E00E946E
:1052C0003B326B01FB01EE0FFF1FEE0FFF1FE4559A
:1052D000FD4FA801012E000C660B770B8081918198
:1052E000A281B381840F951FA61FB71F808391836E
:1052F000A283B38368EB79E082E497E00E94BD1655
:10530000B801CE0101960E947717BE016F5F7F4FF3
:1053100082E497E00E948C16CE0101960E941C1533
:105320006DEA79E088E497E00E94BD16B601CE01EF
:1053300001960E94EE16BE016F5F7F4F88E497E0F2
:105340000E948C16CE0101960E941C1566E072E048
:105350008EE497E00E946D1768E172E084E597E0C3
:105360000E946D1784E090E090938F0280938E02EC
:1053700097CD66E272E082E497E00E946D1765E3E4
:1053800072E088E497E00E946D1767E472E08EE4B3
:1053900097E00E946D1766E572E084E597E00E9451
:1053A0006D1784E090E090938F0280938E020E94AC
:1053B000383027E232E040E050E00E943B32665055
:1053C0007F4F8F4F9F4F60939C0270939D028093FD
:1053D0009E0290939F0264CD5093CD024093CC02E5
:1053E000BCCB0E949E128C01D0928C02C0928B0288
:1053F000F0928A02E092890218161906F4F163E528
:105400007CE082E497E00E94BD1662E57CE088E4DF
:1054100097E00E94BD1662E47CE08EE497E00E9473
:10542000BD166CE37CE084E597E00E94BD166091B8
:10543000890270918A02CE0101960E94EE16BE0189
:105440006F5F7F4F84E597E00E948C16CE01019636
:105450000E941C156AE37CE084E597E00E946216D6
:1054600084E090E090938F0280938E0210928D02E0
:105470008091CC029091CD0263CEF701EE0FFF1F19
:10548000EE0FFF1FEC56FD4FC080D180E280F3800D
:1054900060918502709186028091870290918802C6
:1054A0006C157D058E059F0544F564E37CE082E480
:1054B00097E00E94BD1663E37CE088E497E00E94D9
:1054C000BD1662E27CE08EE497E00E94BD1660911A
:1054D000890270918A02CE0101960E94EE16BE01E9
:1054E0006F5F7F4F84E597E00E940116CE01019621
:1054F0000E941C1560E27CE0AFCF21E130E03093E8
:10550000CD022093CC021092750210927602109276
:105510007702109278020E9408314B015C01C701AA
:10552000B6010E9408319B01AC01C501B4010E9483
:1055300042330E94EA330E94B43360936A0270934C
:105540006B0280936C0290936D02012E000C220B73
:10555000330B06171707280739070CF0FECA00930C
:105560006A0210936B0220936C0230936D02F5CAAD
:1055700084E090E090938C0280938B02F0928A02F8
:10558000E0928902F701EE0FFF1FEE0FFF1FE455B7
:10559000FD4F80819181A281B381181619061A06E8
:1055A0001B06BCF422E130E03093CD022093CC0204
:1055B0001092750210927602109277021092780281
:1055C00080936A0290936B02A0936C02B0936D0279
:1055D000C4CA6AE17CE082E497E00E94BD1669E1FA
:1055E0007CE088E497E00E94BD1666E07CE08EE4F3
:1055F00097E00E94BD166091890270918A02CE01E7
:1056000001960E94EE16BE016F5F7F4F84E597E022
:105610000E940116CE0101960E941C1564E07CE0F8
:105620001BCFD0928C02C0928B0210927502109206
:1056300076021092770210927802E114F10419F1C7
:10564000EA94EF2809F089CA809174028823D1F185
:1056500068EF7BE082E497E00E94BD1669EE7BE094
:1056600088E497E00E94BD1662EE7BE08EE497E04E
:105670000E94BD1683E090E090938F0280938E028B
:1056800010928D020DCC83E190E09093CD02809337
:10569000CC02409185025091860260918702709100
:1056A00088028091810290918202A0918302B09140
:1056B0008402481759076A077B070CF081CFDB018A
:1056C000CA017ECF84E190E09093CD028093CC021A
:1056D000B8E8CB2EB3E1DB2EE12CF12CC0926A02AC
:1056E000D0926B02E0926C02F0926D0236CA85E1B4
:1056F00090E09093CD028093CC02809185029091AE
:105700008602A0918702B09188025ACF84E00E945D
:10571000460F882309F421CA12E0C11AD10825E0F6
:10572000C216D10408F019CA1092D2020E94B41213
:105730009093D1028093D00281E090E033CB81E05E
:105740000E94F41224CA80E00E94F41281111FCA40
:1057500088E00E94460F882309F419CA1092D202E9
:105760008091CC029091CD028C30910509F44EC00D
:1057700060F50B9709F00BCA80917B0290917C0237
:10578000019690937C0280937B0280918502909198
:105790008602A0918702B091880280599140A109A8
:1057A000B1098093850290938602A0938702B093FB
:1057B00088028091790290917A02059790937A02FB
:1057C0008093790281E090E041C08D309105E1F154
:1057D000409709F0DCC98091850290918602A091E2
:1057E0008702B0918802885E9340A109B109809335
:1057F000850290938602A0938702B093880282E389
:1058000090E09093910280939002DCCF8091790296
:1058100090917A020A9690937A028093790280910D
:10582000850290918602A0918702B0918802885CDF
:105830009109A109B1098093850290938602A093F2
:105840008702B0938802BECF8EE090E09093CD02A5
:105850008093CC029CC984E00E94460F8823E1F12A
:105860001092D2020E94383022E030E040E050E056
:105870000E943B32672B682B692BB9F46CE979E005
:1058800082E497E00E94BD1661E979E088E497E040
:105890000E94BD1682E090E090938F0280938E026A
:1058A00010928D0281E090E041C061E879E082E4ED
:1058B00097E00E94BD166BE779E088E497E00E94CC
:1058C000BD1682E090E090938F0280938E0210923A
:1058D0008D0288E090E02AC088E00E94460F88236D
:1058E00009F455C91092D20280917B0290917C02FA
:1058F000892B19F56CE679E082E497E00E94BD16E9
:105900006DE579E088E497E00E94BD1660E579E0F6
:105910008EE497E00E94BD1683E090E090938F02A2
:1059200080938E0210928D0287E090E090938C021B
:1059300080938B028AE090E089CF0E94383022E089
:1059400030E040E050E00E943B32672B682B692B2F
:1059500049F46FE479E082E497E00E94BD166FE3BA
:1059600079E0ABCF8091920290919302019790934E
:10597000930280939202181619064CF46EE379E0B4
:1059800082E497E00E94BD166EE279E096CF0E9415
:10599000383023EE34E040E050E00E943B328B018F
:1059A00002511D4F6CE179E082E497E00E94BD1640
:1059B0006EE079E088E497E00E94BD16B801CE0160
:1059C00001960E947717BE016F5F7F4F88E497E0D2
:1059D0000E948C16CE0101960E941C156CEF78E097
:1059E0008EE497E00E94BD1669EE78E084E597E0CA
:1059F0000E94BD1684E090E090938F0280938E0207
:105A000081E080938D02012E000C220B330B8091DC
:105A1000850290918602A0918702B0918802800F42
:105A2000911FA21FB31F8093850290938602A093BB
:105A30008702B0938802803B9440A105B1050CF425
:105A400031CF80E190E072CF80E00E94F4128111AA
:105A50009EC888E00E94460F882309F43FC18091C8
:105A6000CC029091CD028331910509F4BDC098F428
:105A70008131910509F47FC04297F1F11092D20271
:105A80000E94B4129093D1028093D00280918B0235
:105A900090918C02DBCE8531910509F402C108F4A6
:105AA000CCC0469759F740917502509176026091AB
:105AB00077027091780280917D0290917E02A09190
:105AC0007F02B0918002841B950BA60BB70B8093CD
:105AD0007D0290937E02A0937F02B093800280911A
:105AE000850290918602A0918702B0918802840F6E
:105AF000951FA61FB71F36C08091890290918A0218
:105B0000209175023091760240917702509178028F
:105B1000880F991F880F991FFC01E455FD4FC08025
:105B2000D180E280F380C21AD30AE40AF50AC08267
:105B3000D182E282F3828C569D4FDC016D917D9182
:105B40008D919C910E94943400918502109186025F
:105B50002091870230918802DC01CB01800F911FD8
:105B6000A21FB31F8093850290938602A0938702A1
:105B7000B093880283CF8091890290918A0220910C
:105B80007502309176024091770250917802880F29
:105B9000991F880F991FFC01E455FD4FC080D180EB
:105BA000E280F380C20ED31EE41EF51EC082D182B5
:105BB000E282F3828C569D4FFC016081718182816B
:105BC00093810E9494340091850210918602209165
:105BD00087023091880268017901C61AD70AE80A5B
:105BE000F90AD701C601BECF4091750250917602E5
:105BF0006091770270917802809181029091820287
:105C0000A0918302B0918402841B950BA60BB70B65
:105C10008093810290938202A0938302B0938402C6
:105C20008091850290918602A0918702B0918802AE
:105C3000841B950BA60BB70B95CF40917502509125
:105C40007602609177027091780280918102909142
:105C50008202A0918302B0918402840F951FA61F37
:105C6000B71F8093810290938202A0938302B09326
:105C700084028091850290918602A0918702B09162
:105C80008802840F951FA61FB71F809385029093EB
:105C90008602A0938702B093880281E08093740209
:105CA000EDCE40917502509176026091770270912D
:105CB000780280917D0290917E02A0917F02B09146
:105CC0008002840F951FA61FB71F80937D029093BB
:105CD0007E02A0937F02B0938002A2CF8FB7F89488
:105CE0004090D4025090D5026090D6027090D702B6
:105CF0008FBF8091CC029091CD024197C12CD12CC5
:105D00007601C394029728F07AE0C72ED12CE12CBB
:105D1000F12C8091700290917102A0917202B09169
:105D2000730293018201081B190B2A0B3B0B809114
:105D30006E0290916F0244EF51E060E070E08230BB
:105D4000910554F044E650E060E070E08531910543
:105D50001CF040E050E0BA0140175107620773079A
:105D600010F00C94C725843691050CF45EC05AE0FF
:105D7000852E912CA12CB12C8D379105BCF044E6D9
:105D8000842E912CA12CB12C863991057CF068EEE3
:105D9000862E63E0962EA12CB12C8F3A910534F01B
:105DA00030E1832E37E2932EA12CB12C883E03E004
:105DB00090072CF4019690936F0280936E0280E816
:105DC0000E94510F882309F441C040927002509202
:105DD0007102609272027092730240916A02509155
:105DE0006B0260916C0270916D02809175029091CE
:105DF0007602A0917702B09178028A019B010C197A
:105E00001D092E093F09081719072A073B0794F0B7
:105E10008C0D9D1DAE1DBF1D809375029093760263
:105E2000A0937702B09378020DC0812C912C54017D
:105E30008394C0CF409375025093760260937702AB
:105E4000709378020E94D0140C94C72580E40E94BD
:105E5000510F8823C9F140927002509271026092F2
:105E6000720270927302AAE0B0E0A70196010E944C
:105E70005A329B01AC01C501B4010E9494340091D7
:105E80007502109176022091770230917802DC0140
:105E9000CB01800F911FA21FB31F00916A021091C6
:105EA0006B0220916C0230916D02081719072A07C6
:105EB0003B070CF0B1CF009375021093760220934C
:105EC000770230937802BECF80E10E94510F882381
:105ED00019F14092700250927102609272027092B7
:105EE00073028091750290917602A0917702B09131
:105EF00078028C159D05AE05BF052CF08C199D0907
:105F0000AE09BF0989CF10927502109276021092E5
:105F100077021092780296CF80E20E94510F882378
:105F200051F140927002509271026092720270922E
:105F30007302AAE0B0E0A70196010E945A329B01C9
:105F4000AC01C501B4010E94943400917502109116
:105F500076022091770230917802061717072807FA
:105F600039078CF268017901C61AD70AE80AF90ADA
:105F7000D701C60151CF1092700210927102109297
:105F800072021092730210926F0210926E020C94C1
:105F9000C725CF93DF938AE597E00E941C1584E51F
:105FA00097E00E941C158EE497E00E941C1588E47F
:105FB00097E00E941C1582E497E00E941C15C4E83B
:105FC000D7E02697CE010E941C1587E0C036D8077F
:105FD000C1F7DF91CF9108958F929F92AF92BF92B8
:105FE000CF92DF92EF92FF92CF93DF93EC01688123
:105FF00079818A819B81611571058105910521F463
:1060000064E279ED8BE597E02DE133EF41E050E07C
:106010000E943B3249015A019B01AC01A7EAB1E45D
:106020000E945A326B017C01ACEEB4EFA5019401E1
:106030000E946832C60ED71EE81EF91EF7FE06C083
:1060400081E0C81AD108E10880E8F80AC882D9823C
:10605000EA82FB82C701B6019F77DF91CF91FF9063
:10606000EF90DF90CF90BF90AF909F908F9008956A
:106070008F929F92AF92BF92CF92DF92EF92FF9258
:1060800060910D0170910E0180910F0190911001AE
:10609000611571058105910521F464E279ED8BE5C7
:1060A00097E02DE133EF41E050E00E943B3249019F
:1060B0005A019B01AC01A7EAB1E40E945A326B017C
:1060C0007C01ACEEB4EFA50194010E946832C60ECB
:1060D000D71EE81EF91EF7FE06C081E0C81AD108D7
:1060E000E10880E8F80AC0920D01D0920E01E0921A
:1060F0000F01F0921001C701B6019F77FF90EF905A
:10610000DF90CF90BF90AF909F908F900895609355
:106110000D0170930E0180930F019093100108956B
:10612000FB01DC0105900D920020E1F70895FC01D0
:1061300005900020E9F7809590958E0F9F1F089598
:10614000BB274A3031F4992322F4BDE29095819522
:106150009F4F0C94DD30BB272A3051F4992342F431
:10616000BDE290958095709561957F4F8F4F9F4FC1
:106170000C94BB30BB27FA01A62F6217710581056D
:106180009105330B30FB66F0AA27660F771F881F37
:10619000991FAA1FA21710F0A21B63953850A9F7E8
:1061A000A05DAA3308F0A95DA19336F7B111B193B0
:1061B0001082CA010C94F630BB27FB015527AA2791
:1061C000880F991FAA1FA41710F0A41B8395505184
:1061D000B9F7A05DAA3308F0A95DA193009779F7FC
:1061E000B111B1931192CB010C94F630DC01FC019A
:1061F000672F71917723E1F7329704C07C916D93FB
:1062000070836291AE17BF07C8F30895E89409C080
:1062100097FB3EF490958095709561957F4F8F4FD9
:106220009F4F9923A9F0F92F96E9BB279395F695EF
:10623000879577956795B795F111F8CFFAF4BB0F6D
:1062400011F460FF1BC06F5F7F4F8F4F9F4F16C0D1
:10625000882311F096E911C0772321F09EE8872F5B
:10626000762F05C0662371F096E8862F70E060E017
:106270002AF09A95660F771F881FDAF7880F969590
:10628000879597F90895990F0008550FAA0BE0E834
:10629000FEEF16161706E807F907C0F012161306E8
:1062A000E407F50798F0621B730B840B950B39F428
:1062B0000A2661F0232B242B252B21F408950A268E
:1062C00009F4A140A6958FEF811D811D08950E94BC
:1062D0007A310C94EB310E94DD3138F00E94E431C8
:1062E00020F0952311F00C94D4310C94DA31112460
:1062F0000C941F320E94FC3170F3959FC1F3950FEF
:1063000050E0551F629FF001729FBB27F00DB11D39
:10631000639FAA27F00DB11DAA1F649F6627B00DC9
:10632000A11D661F829F2227B00DA11D621F739FB2
:10633000B00DA11D621F839FA00D611D221F749FC0
:106340003327A00D611D231F849F600D211D822F07
:10635000762F6A2F11249F5750409AF0F1F088232E
:106360004AF0EE0FFF1FBB1F661F771F881F91505B
:106370005040A9F79E3F510580F00C94D4310C9405
:106380001F325F3FE4F3983ED4F386957795679587
:10639000B795F795E7959F5FC1F7FE2B880F911D85
:1063A0009695879597F9089597F99F6780E870E02B
:1063B00060E008959FEF80EC089500240A9416167B
:1063C000170618060906089500240A9412161306E3
:1063D000140605060895092E0394000C11F4882371
:1063E00052F0BB0F40F4BF2B11F460FF04C06F5F8D
:1063F0007F4F8F4F9F4F089557FD9058440F551F63
:1064000059F05F3F71F04795880F97FB991F61F036
:106410009F3F79F087950895121613061406551FAD
:10642000F2CF4695F1DF08C0161617061806991F19
:10643000F1CF86957105610508940895E894BB270E
:1064400066277727CB0197F90895F999FECF92BD7A
:1064500081BDF89A992780B50895262FF999FECF26
:106460001FBA92BD81BD20BD0FB6F894FA9AF99A71
:106470000FBE01960895052E97FB1EF400940E940E
:10648000523257FD07D00E94A43207FC03D04EF4CD
:106490000C94523250954095309521953F4F4F4F77
:1064A0005F4F089590958095709561957F4F8F4FC0
:1064B0009F4F08950E94C632A59F900DB49F900DE6
:1064C000A49F800D911D11240895B7FF0C945A329A
:1064D0000E945A32821B930B08952F923F924F9243
:1064E0005F926F927F928F929F92AF92BF92CF9264
:1064F000DF92EF92FF920F931F93CF93DF93CDB76D
:10650000DEB7CA1BDB0B0FB6F894DEBF0FBECDBFE4
:1065100009942A88398848885F846E847D848C84B5
:106520009B84AA84B984C884DF80EE80FD800C81BE
:106530001B81AA81B981CE0FD11D0FB6F894DEBFA1
:106540000FBECDBFED010895A1E21A2EAA1BBB1B01
:10655000FD010DC0AA1FBB1FEE1FFF1FA217B3072F
:10656000E407F50720F0A21BB30BE40BF50B661F45
:10657000771F881F991F1A9469F760957095809509
:1065800090959B01AC01BD01CF010895A29FB00180
:10659000B39FC001A39F700D811D1124911DB29F57
:1065A000700D811D1124911D08955058BB27AA27F5
:1065B0000E94ED320C94EB310E94DD3138F00E94E4
:1065C000E43120F039F49F3F19F426F40C94DA31C9
:1065D0000EF4E095E7FB0C94D431E92F0E94FC31D6
:1065E00058F3BA17620773078407950720F079F408
:1065F000A6F50C941E320EF4E0950B2EBA2FA02DAA
:106600000B01B90190010C01CA01A0011124FF275F
:10661000591B99F0593F50F4503E68F11A16F0405A
:10662000A22F232F342F4427585FF3CF4695379559
:106630002795A795F0405395C9F77EF41F16BA0B1E
:10664000620B730B840BBAF09150A1F0FF0FBB1FCC
:10665000661F771F881FC2F70EC0BA0F621F731F15
:10666000841F48F4879577956795B795F7959E3F72
:1066700008F0B0CF9395880F08F09927EE0F979503
:10668000879508950E9456330C94EB310E94E431B3
:1066900058F00E94DD3140F029F45F3F29F00C945E
:1066A000D43151110C941F320C94DA310E94FC3118
:1066B00068F39923B1F3552391F3951B550BBB2731
:1066C000AA2762177307840738F09F5F5F4F220F76
:1066D000331F441FAA1FA9F335D00E2E3AF0E0E86D
:1066E00032D091505040E695001CCAF72BD0FE2FB7
:1066F00029D0660F771F881FBB1F2617370748074B
:10670000AB07B0E809F0BB0B802DBF01FF27935802
:106710005F4F3AF09E3F510578F00C94D4310C94C1
:106720001F325F3FE4F3983ED4F3869577956795E3
:10673000B795F7959F5FC9F7880F911D9695879537
:1067400097F90895E1E0660F771F881FBB1F621756
:1067500073078407BA0720F0621B730B840BBA0B14
:10676000EE1F88F7E09508950E94BB336894B1113D
:106770000C941F3208950E94043288F09F5798F0BD
:10678000B92F9927B751B0F0E1F0660F771F881F36
:10679000991F1AF0BA95C9F714C0B13091F00E9450
:1067A0001E32B1E008950C941E32672F782F88278F
:1067B000B85F39F0B93FCCF3869577956795B39577
:1067C000D9F73EF490958095709561957F4F8F4FE6
:1067D0009F4F08950E942A3490F09F3748F49111FA
:1067E00016F00C941F3260E070E080E89FEB089593
:1067F00026F41B16611D711D811D0C9401340C942F
:106800001C34882371F4772321F09850872B762F3E
:1068100007C0662311F499270DC09051862B70E0B4
:1068200060E02AF09A95660F771F881FDAF7880FC5
:106830009695879597F908959F3F31F0915020F4F0
:10684000879577956795B795880F911D969587954C
:1068500097F908950E940432A0F0BEE7B91788F4B2
:10686000BB279F3860F41616B11D672F782F882735
:10687000985FF7CF869577956795B11D9395963973
:10688000C8F308950E94433108F48FEF089519F476
:1068900016F40C94DA310C941C340E940432B8F3D0
:1068A0009923C9F3B6F39F57550B87FF0E948D3488
:1068B0000024A0E640EA900180585695979528F468
:1068C000805C660F771F881F20F026173707480760
:1068D00030F4621B730B840B202931294A2BA695B7
:1068E00017940794202531254A2758F7660F771FFC
:1068F000881F20F026173707480730F4620B730B08
:10690000840B200D311D411DA09581F7B901842F05
:106910009158880F96958795089591505040660F2D
:10692000771F881FD2F70895DB018F939F930E94F2
:106930005A32BF91AF91A29F800D911DA39F900DE0
:10694000B29F900D11240895EE0FFF1F0590F49152
:10695000E02D09940F931F93CF93DF93823091051D
:1069600010F482E090E0E0919E07F0919F0730E004
:1069700020E0B0E0A0E0309799F42115310509F44A
:106980004AC0281B390B24303105D8F58A819B81F8
:106990006115710589F1FB0193838283FE0111C0AA
:1069A000408151810281138148175907E0F048174F
:1069B000590799F4109761F012960C931297139659
:1069C0001C933296CF01DF91CF911F910F910895C3
:1069D00000939E0710939F07F4CF2115310551F0C6
:1069E0004217530738F0A901DB019A01BD01DF010D
:1069F000F801C1CFEF01F9CF90939F0780939E07D5
:106A0000CDCFFE01E20FF31F819391932250310904
:106A100039832883D7CF20919C0730919D07232B62
:106A200041F4209113013091140130939D0720937C
:106A30009C0720911101309112012115310541F47B
:106A40002DB73EB74091150150911601241B350B0F
:106A5000E0919C07F0919D07E217F307A0F42E1B2D
:106A60003F0B2817390778F0AC014E5F5F4F2417B2
:106A7000350748F04E0F5F1F50939D0740939C07CA
:106A8000819391939FCFF0E0E0E09CCFCF93DF9391
:106A90000097E9F0FC01329713821282A0919E07C1
:106AA000B0919F07ED0130E020E01097A1F4208124
:106AB0003181820F931F20919C0730919D072817E9
:106AC000390709F061C0F0939D07E0939C07DF91BF
:106AD000CF910895EA01CE17DF07E8F54A815B817F
:106AE0009E0141155105B1F7E901FB83EA83499104
:106AF0005991C40FD51FEC17FD0761F48081918176
:106B00000296840F951FE90199838883828193817E
:106B10009B838A83F0E0E0E012968D919C9113971D
:106B20000097B9F52D913C911197CD010296820FF6
:106B3000931F20919C0730919D072817390739F63C
:106B4000309751F510929F0710929E07B0939D07C2
:106B5000A0939C07BCCFD383C28340815181840F13
:106B6000951FC817D90761F44E5F5F4F88819981DF
:106B7000480F591F518340838A819B81938382836D
:106B80002115310509F0B0CFF0939F07E0939E07E0
:106B90009ECFFD01DC01C0CF13821282D7CFB0E0BF
:106BA000A0E0E5EDF5E30C946F328C01009751F411
:106BB000CB010E94AA348C01C801CDB7DEB7E0E159
:106BC0000C948B32FC01E60FF71F9C012250310917
:106BD000E217F30708F49DC0D901CD91DC9111971C
:106BE000C617D70798F0C530D10530F3CE0104970A
:106BF0008617970708F3C61BD70B2297C193D1932B
:106C00006D937C93CF010E944635D6CF5B01AC1AC1
:106C1000BD0A4C018C0E9D1EA0919E07B0919F074E
:106C2000512C412CF12CE12C109731F580919C07CF
:106C300090919D078815990509F05CC04616570686
:106C400008F058C08091110190911201009741F411
:106C50008DB79EB74091150150911601841B950B7D
:106C6000E817F90708F055C0F0939D07E0939C07DB
:106C7000F90171836083A0CF8D919C911197129639
:106C80006C90129713967C901397A815B90559F537
:106C90006C0142E0C40ED11CCA14DB0420F1AC012B
:106CA0004A195B09DA011296159780F062827382A5
:106CB00051834083D9016D937C93E114F10471F009
:106CC000D7011396FC93EE93129776CF22968C0FF2
:106CD0009D1FF90191838083F301EFCFF0939F070C
:106CE000E0939E0769CF4816590608F42C017D01F0
:106CF000D3019ACFCB010E94AA347C01009749F0BE
:106D0000AE01B8010E948C36C8010E944635870149
:106D100053CF10E000E050CFFB01DC0102C0019036
:106D20000D9241505040D8F70895FB01DC010190CD
:106D30000D920020E1F7089517E0C1EBD7E004C001
:106D4000FE010E94A4342196C23BD107C9F7F894F2
:026D5000FFCF73
:106D520010FFFFFFFF00E100000000000001000043
:106D6200000000A007800000C18081000000000038
:106D72000000F50B600D160C0B0C5C0C1A0C380C99
:106D8200000000005012CA0EC313E50D00000000FF
:106D92000212CA0EC313E50D00000000CA10CA0E8B
:106DA200C313E50D596F75206F776E2000596F750B
:106DB2002065617420697420616C6C2062757400B6
:106DC200666F7267657420746F20627275736820D3
:106DD200796F75720074656574682E2054686579E0
:106DE20020616C6C20726F7400616E6420796F7523
:106DF2002063616E27742065617400736F6C69642F
:106E020020666F6F6420616E796D6F72652E00204F
:106E120020204A75737420736179206E6F002020E0
:106E22002020746F2063616E64792E0020204761F8
:106E32006D65206F76657221002020596F75722072
:106E420073636F72653A200020206F7574206F663D
:106E5200203130302E00696E2061206C756E6368BF
:106E620020626F7820696E0074686520737562779E
:106E7200617921212100546865206D61726B65740E
:106E820020686173006265656E20666C6F6F646571
:106E920064207769746800636865617020686F6D4B
:106EA200656D616465004165726F212121210000D9
:00000001FF
